:0400000057EF00F0C6
:100008002B002B002B002B002B002B002B002B0090
:100018002B002B002B002B002B002B002B002B0080
:100028002B002B002B002B002B002B002B002B0070
:100038002B002B002B006C532B002B002B002B00CC
:1000480097572B002B002B002B002B002B002B008D
:100058002B002B002B002B002B002B002B002B0040
:100068002B002B002B002B002B002B002B002B0030
:100078002B002B002B002B002B002B002B002B0020
:100088002B002B002B002B002B002B002B002B0010
:10009800E3552B002B002B002B002B002B002B00F3
:0A00A8002B002B00FF0040EFA8F032
:10FAA60000000000001B1B1B1B1B1B1B1B00000078
:10FAB600000303030318181818181818180303036B
:10FAC600030000001F1F1F1F1F00001F1F1F1F1FF7
:10FAD6001F001F1F1F1F1F1F1F1F1F1F1F1F1F1F4F
:10FAE6001F8080808080808080C0C0C0C0C0C0C0B1
:10FAF600C0E0E0E0E0E0E0E0E0F0F0F0F0F0F0F0B0
:10FB0600F0F8F8F8F8F8F8F8F8FCFCFCFCFCFCFC5B
:10FB1600FCFEFEFEFEFEFEFEFEFFFFFFFFFFFFFFFA
:10FB2600FF0C12120C000000000609081E1E080930
:10FB360006040A11110A0A1100040E0E0E1F000413
:10FB4600001C141B12131212000103070F070301F6
:10FB56000000110A0406110000000103161C100023
:10FB6600004C63013E6001766201B43D01104D0117
:10FB76000051016C4C013E6301EA6301E663011624
:10FB860061019263019A63013063018A6301206314
:10FB9600012E550168530110630170507700070468
:10FBA60004070080C094D420200020446972656355
:10FBB600746F7279203A433A5C4D504C4142585F1B
:10FBC60050726F6A656374735C5F31384632374BC7
:10FBD60034325F4F57535F445331384232305F32CD
:10FBE6003032332E580D0A005A65726F2020007588
:10FBF6006E20202020006465757820200074726FC6
:10FC0600697320007175617472650063696E712095
:10FC1600200073697820202000536570742020002E
:10FC2600444547524545004555524F2020004F4810
:10FC36004D202020005046202020200044726F696D
:10FC46007465004761756368650043414E43454CE2
:10FC560000436865636B2E002050494331384632B5
:10FC6600374B3432202B204F57532073656E736FFA
:10FC7600722044533138423230207375722020503E
:10FC86004F525420524130290D0A0020417574729A
:10FC96006573203A2020445331384232305F626126
:10FCA600726B65722E6820204F6E65576972655FAC
:10FCB6006261726B65722E680D0A00205241303DFA
:10FCC60044533138423230205241343D6C65642011
:10FCD600205241333D535141205243363D54582022
:10FCE60055415254310D0A002050726F6A65637493
:10FCF600203A202031384632374B34325F4F575343
:10FD06005F445331384232305F323032330D0A00AD
:10FD160020436F6E6669672020496E7465726E6156
:10FD26006C20466F73632036344D487A0D0A0020E6
:10FD3600536F75726365203A20206D61696E2E637C
:10FD4600205F323032332D303430370D0A00202018
:10FD560020202020202020202020202020200020BD
:10FD6600456570726F6D203A204E6F6E0D0A002049
:10FD7600002000204020646563696D616C202325A6
:10FD860034752020736F6974204044657669636515
:10FD9600203762697473203D203058253032582050
:10FDA600002054657374207072E973656E63652074
:10FDB6006427756E2063617074657572204F2E57C7
:10FDC6002E532E20737572205241300D0A00205496
:10FDD6006573742070726573656E636520646576FD
:10FDE60069636573207375722042757320493243C7
:10FDF600310D0A00200D0A496E69742032204C43E9
:10FE060044204932432076696120504346383735CD
:10FE1600340D0A00200D0A20436F6E66696720655F
:10FE26007420496E6974204F6E6520576972650D9E
:10FE36000A002025303564202074656D70203D2031
:10FE460025352E33662025632043200D0A002041E8
:10FE5600666669636861676520737572204C434402
:10FE66002032783136200D0A0020436F6465204623
:10FE7600616D696C6C65203A2044533138423230EA
:10FE86000D0A002061647265737365204C43443D1E
:10FE9600202564202025303278200D0A002050438A
:10FEA600463837353420666F72204C43442032780A
:10FEB60031366361727300204D6573757265204437
:10FEC600533138423230202331203A200D0A0020A7
:10FED600202020202020202020202020202020201C
:10FEE60020202000202053656E736F7220446174B9
:10FEF6006173203A0D0A00504346383537344120A5
:10FF0600386269747320492F4F004C4344203231C4
:10FF1600313920327831366361727300542E455878
:10FF26005445522E2020202020202020003132331C
:10FF3600343536373839303132333435360050437C
:10FF4600463835373420386269747320494F00418A
:10FF560042434445464748494A4B4C4D4E4F500054
:10FF66002050726573656E746174696F6E203A0015
:10FF7600454550524F4D20353132627974657300D4
:10FF860020435243203D2025303258200D0A0020C0
:10FF9600496E69745F49324328293B0D0A004F4C6C
:10FFA6004544205353443133303600204F575320B5
:10FFB600494423203D20006E6F6E20726563656E96
:10FFC60073E9005254432044533332333100303006
:10FFD600302E303020430025332E32662043002554
:10FFE6003032582E00494E46004E414E00696E662C
:09FFF600006E616E006C660000F3
:020000040001F9
:10000000000E0001756F000E746F36C086F037C0A9
:1000100087F038C088F039C089F089BF14EF80F0CC
:1000200012EF80F02AEF80F0000E756F010E746FF2
:1000300086C001F087C002F088C003F089C004F0D8
:10004000F6ECAEF001C086F002C087F003C088F085
:1000500004C089F0000E00018D6F000E8C6FC6C0C9
:1000600078F0C7C079F074517511D8A43AEF80F0D8
:100070003CEF80F043EF80F0CAA541EF80F043EF02
:1000800080F05DEF80F074517511D8A44AEF80F0D4
:100090004CEF80F052EF80F0000E616F2B0E606F1E
:1000A00056EF80F0000E616F2D0E606F60C06CF136
:1000B0008C4B8D2B7807D8A0790786C001F087C0BC
:1000C00002F088C003F089C004F072ECA0F00104D3
:1000D0000210D8A46EEF80F070EF80F0BBEF80F0DC
:1000E000BF0E3B6EFF0E3C6E3A503D6E3E6A3B507B
:1000F0003D263C503E223E5007E11A0E3D5CD8B0F2
:1001000084EF80F086EF80F095EF80F06C0E0001B8
:100110008C25056E010E8D21066EEB0E076EFF0E0F
:10012000086E03ECABF0A2EF80F06C0E00018C25A2
:10013000056E010E8D21066EF30E076EFF0E086E22
:1001400003ECABF00001FD0E7827FF0E792334C0DD
:1001500011F035C012F06C0E136E010E146E78C0E3
:1001600015F079C016F012ECA4F011C034F012C0F2
:1001700035F008EF86F086C001F087C002F088C035
:1001800003F089C004F072ECA0F001500210D8A472
:10019000CCEF80F0CEEF80F002EF81F0BF0E3B6E2F
:1001A000FF0E3C6E3A503D6E3E6A3B503D263C5041
:1001B0003E223E5007E11A0E3D5CD8B0E2EF80F0DF
:1001C000E4EF80F0F3EF80F06C0E00018C25056EFB
:1001D000010E8D21066EEF0E076EFF0E086E03EC0A
:1001E000ABF0A2EF80F06C0E00018C25056E010EC5
:1001F0008D21066EF70E076EFF0E086E03ECABF056
:10020000A2EF80F0000E00018E6F000E8F6F800E47
:10021000906F3F0E916F000E8B6F000E8A6F86C03D
:1002200001F087C002F088C003F089C004F0000E1E
:10023000056E000E066E000E076E000E086E8FEC47
:10024000A5F0D8B026EF81F028EF81F0ABEF81F078
:1002500047EF81F08EC00FF08FC010F090C011F00A
:1002600091C012F0000E136E000E146E200E156E6B
:10027000410E166EB6EC8DF00FC08EF010C08FF0F0
:1002800011C090F012C091F000018A4B8B2B86C0F8
:1002900028F087C029F088C02AF089C02BF0000E12
:1002A000136E000E146E200E156E410E166E8EC06B
:1002B0000FF08FC010F090C011F091C012F0B6ECAA
:1002C0008DF00FC02CF010C02DF011C02EF012C018
:1002D0002FF0F0EC9FF0D8B070EF81F072EF81F06A
:1002E0002AEF81F092EF81F08EC001F08FC002F012
:1002F00090C003F091C004F0000E056E000E066E73
:10030000200E076E410E086EDDEC8FF001C08EF0FE
:1003100002C08FF003C090F004C091F000018A0782
:10032000D8A08B0786C028F087C029F088C02AF0A3
:1003300089C02BF08EC02CF08FC02DF090C02EF015
:1003400091C02FF0F0EC9FF0D8A0A9EF81F0ABEFB7
:1003500081F074EF81F03AC007F0086A5DECADF00F
:10036000075000017B6F7BC07AF0670E7B19D8A421
:10037000BCEF81F0BEEF81F0E4EF81F0C851C9110C
:10038000D8A4C5EF81F0C7EF81F0CBEF81F0000E6C
:10039000C96F010EC86FC9BFD8EF81F0C95106E11E
:1003A000C805D8B0D6EF81F0D8EF81F0DEEF81F04C
:1003B000000E776F060E766FEDEF81F0C8C076F015
:1003C000C9C077F0EDEF81F0C9BFE9EF81F0EBEF45
:1003D00081F0D8EF81F0DEEF81F0670E7B19D8A4B1
:1003E000F4EF81F0F6EF81F025EF82F08BAF04EFB0
:1003F00082F0FC0E8A5DFF0E8B59D8A002EF82F0CE
:1004000004EF82F023EF82F0FF0E3B6EFF0E3C6E96
:1004100076C03DF077C03EF03B503D263C503E223A
:100420008A513D5C3E50800A3F6E8B51800A3F5896
:10043000D8A01DEF82F01FEF82F023EF82F0660E4E
:100440007A6F25EF82F0650E7A6F76C06CF077C018
:100450006DF0670E7B19D8A430EF82F032EF82F096
:1004600042EF82F0660E7A19D8A439EF82F03BEFA2
:1004700082F044EF82F08BBF42EF82F040EF82F0D7
:1004800044EF82F06C4B6D2B660E7A19D8A44BEFBB
:1004900082F04DEF82F06DEF82F08BBF54EF82F06F
:1004A00052EF82F060EF82F0000E8E6F000E8F6FC1
:1004B000800E906F3F0E916F000E8B6F000E8A6F53
:1004C000670E7B19D8B467EF82F069EF82F06DEFA9
:1004D00082F08A516C278B516D23000E856F000EC0
:1004E000846F86C07CF087C07DF088C07EF089C0B4
:1004F0007FF08EC06EF08FC06FF090C070F091C032
:1005000071F0FEEF82F07CC001F07DC002F07EC091
:1005100003F07FC004F08EC005F08FC006F090C0DD
:1005200007F091C008F0DDEC8FF001C01AF002C0B6
:100530001BF003C01CF004C01DF019EC99F01AC0A8
:1005400080F01BC081F01CC082F01DC083F080C011
:1005500001F081C002F082C003F083C004F06DECB2
:100560009FF001C072F002C073F07CC028F07DC023
:1005700029F07EC02AF07FC02BF08EC013F08FC010
:1005800014F090C015F091C016F080C00FF081C03B
:1005900010F082C011F083C012F0B6EC8DF00FC0E5
:1005A0002CF010C02DF011C02EF012C02FF080ECF6
:1005B000ADF028C07CF029C07DF02AC07EF02BC0B1
:1005C0007FF08EC001F08FC002F090C003F091C0A8
:1005D00004F0000E056E000E066E200E076E410E32
:1005E000086EDDEC8FF001C08EF002C08FF003C00A
:1005F00090F004C091F00001844B852B6C51845D18
:100600008551800A3B6E6D51800A3B58D8A00BEF94
:1006100083F00DEF83F083EF82F08EC00FF08FC078
:1006200010F090C011F091C012F0000E136E000E89
:10063000146EA00E156E400E166EB6EC8DF00FC047
:1006400080F010C081F011C082F012C083F07CC035
:1006500028F07DC029F07EC02AF07FC02BF080C03A
:100660002CF081C02DF082C02EF083C02FF0F0EC72
:100670009FF0D8B03EEF83F040EF83F04BEF83F074
:10068000000E0001806F000E816F000E826F000E61
:10069000836F74EF83F07CC001F07DC002F07EC0F8
:1006A00003F07FC004F080C005F081C006F082C076
:1006B00007F083C008F08FECA5F0D8A062EF83F0BC
:1006C00064EF83F074EF83F0000172B16AEF83F09E
:1006D0006CEF83F074EF83F0000E806F000E816F7B
:1006E000000E826F000E836F86C001F087C002F09B
:1006F00088C003F089C004F080C005F081C006F016
:1007000082C007F083C008F056EC8BF001C07CF08B
:1007100002C07DF003C07EF004C07FF07CC028F0F2
:100720007DC029F07EC02AF07FC02BF0000E136E32
:10073000000E146E200E156E410E166E6EC00FF078
:100740006FC010F070C011F071C012F0B6EC8DF0F7
:100750000FC02CF010C02DF011C02EF012C02FF0E1
:10076000F0EC9FF0D8A0B7EF83F0B9EF83F0E2EFA1
:1007700083F000018A4B8B2B6EC00FF06FC010F01E
:1007800070C011F071C012F0000E136E000E146EE6
:10079000200E156E410E166EB6EC8DF00FC06EF089
:1007A00010C06FF011C070F012C071F0660E000141
:1007B0007A19D8A4DEEF83F0E0EF83F0E2EF83F064
:1007C0006C4B6D2B6EC08EF06FC08FF070C090F0D0
:1007D00071C091F0650E00017A19D8B4F2EF83F080
:1007E000F4EF83F0FAEF83F08AC06AF08BC06BF00D
:1007F000FEEF83F0000E6B6F000E6A6F000E696FE4
:10080000000E686F000E676F000E666F000E856F3A
:10081000000E846FF9EF84F07CC001F07DC002F01F
:100820007EC003F07FC004F08EC005F08FC006F0DC
:1008300090C007F091C008F0DDEC8FF001C01AF015
:1008400002C01BF003C01CF004C01DF019EC99F0AD
:100850001AC080F01BC081F01CC082F01DC083F064
:1008600080C001F081C002F082C003F083C004F0B8
:100870006DEC9FF001C072F002C073F00001CAB9C4
:1008800044EF84F046EF84F063EF84F0725173110B
:10089000D8A44DEF84F04FEF84F063EF84F0670E3F
:1008A0007B19D8A456EF84F058EF84F063EF84F0FE
:1008B0006BBF5FEF84F05DEF84F063EF84F0664B15
:1008C000672BADEF84F068516911D8A46AEF84F00A
:1008D0006CEF84F096EF84F06BBF73EF84F071EFF0
:1008E00084F096EF84F06C0E8C25D96E010E8D216C
:1008F000DA6E2E0EDF6E8C4B8D2B7807D8A0790721
:10090000000E696F010E686F96EF84F06C0E8C25F7
:10091000D96E010E8D21DA6E300EDF6E8C4B8D2B71
:100920007807D8A079076607D8A0670766516711CE
:10093000D8A49DEF84F09FEF84F086EF84F06C0ED6
:100940008C25D96E010E8D21DA6E7251300FDF6E5B
:100950008C4B8D2B7807D8A079077CC028F07DC000
:1009600029F07EC02AF07FC02BF08EC013F08FC01C
:1009700014F090C015F091C016F080C00FF081C047
:1009800010F082C011F083C012F0B6EC8DF00FC0F1
:100990002CF010C02DF011C02EF012C02FF080EC02
:1009A000ADF028C07CF029C07DF02AC07EF02BC0BD
:1009B0007FF08EC001F08FC002F090C003F091C0B4
:1009C00004F0000E056E000E066E200E076E410E3E
:1009D000086EDDEC8FF001C08EF002C08FF003C016
:1009E00090F004C091F000016A07D8A06B07844B17
:1009F000852B6C51845D8551800A3B6E6D51800A58
:100A00003B58D8B006EF85F008EF85F016EF85F07B
:100A10008DBF14EF85F08D5109E14B0E8C5DD8A090
:100A200014EF85F016EF85F00CEF84F06851691132
:100A3000D8A41DEF85F01FEF85F030EF85F0CAA92F
:100A400024EF85F026EF85F030EF85F06C0E8C25D5
:100A5000D96E010E8D21DA6E2E0EDF6E8C4B8D2B32
:100A60006C0E8C25D96E010E8D21DA6E000EDF6EB4
:100A7000650E7A19D8A43FEF85F041EF85F0A7EF16
:100A800080F0000E856F4F0E846F6C0E8425D96E3A
:100A9000010E8521DA6E000EDF6E000E756F000EFE
:100AA000746F8BBF58EF85F056EF85F060EF85F0DF
:100AB000000E756F010E746F8A6D8B1FD8B08B2B73
:100AC000000E776F020E766F91EF85F08407D8A045
:100AD00085076C0E8425D96E010E8521DA6E8AC0D9
:100AE00001F08BC002F0000E046E0A0E036E37ECAC
:100AF000A5F00150300FDF6E8AC001F08BC002F00C
:100B0000000E046E0A0E036E75ECA4F001C08AF0AC
:100B100002C08BF000017607D8A077077807D8A02D
:100B200079078A518B11D8A498EF85F09AEF85F058
:100B300066EF85F077BFA7EF85F0775106E1760580
:100B4000D8B0A5EF85F0A7EF85F066EF85F08407B4
:100B5000D8A0850774517511D8A4B1EF85F0B3EF13
:100B600085F0B9EF85F0000E636F2B0E626FBDEF5D
:100B700085F0000E636F2D0E626F6C0E8425D96EAA
:100B8000010E8521DA6E60008BF1DFFF7807D8A0B7
:100B900079078407D8A08507BF0E3B6EFF0E3C6E19
:100BA0003A503D6E3E6A3B503D263C503E223E5000
:100BB00009E11A0E3D5CD8A0E0EF85F0E2EF85F088
:100BC000E8EF85F0000E656F650E646FECEF85F061
:100BD000000E656F450E646F6C0E8425D96E010E94
:100BE0008521DA6E600093F1DFFF7807D8A07907DE
:100BF0006C0E8C25056E010E8D21066E6C0E842503
:100C0000076E010E8521086E03ECABF0A7EF80F0B4
:100C1000120060000BF1D9FF60000FF1DAFF6F00E6
:100C20007BFFF6FF6F0077FFF7FF000EF86E0800FE
:100C3000F550250AD8A41FEF86F021EF86F032EF99
:100C40008BF060000BF1D9FF60000FF1DAFFDE2AB4
:100C5000000EDD22000E0001C76F000EC66FC6C079
:100C6000CAF0C7C0CBF0C869C969000E9B6F000EFF
:100C70009A6F89EF86F0CA8160000BF1D9FF60009E
:100C80000FF1DAFFDE2A000EDD2289EF86F0CA833B
:100C90003CEF86F0CA853CEF86F0CA873CEF86F0D1
:100CA000CA893CEF86F0000E9B6F010E9A6F89EFA8
:100CB00086F060000BF1D9FF60000FF1DAFF6F00E2
:100CC0007BFFF6FF6F0077FFF7FF000EF86E08005E
:100CD000F550466E476A4750000AD8B472EF86F066
:100CE00053EF86F04650200AD8B44DEF86F0030A41
:100CF000D8B450EF86F0080AD8B44AEF86F0060A56
:100D0000D8B43BEF86F01D0AD8B447EF86F053EF16
:100D100086F09A519B11D8B490EF86F092EF86F04E
:100D200059EF86F0CAA197EF86F099EF86F09AEF17
:100D300086F0CA9360000BF1D9FF60000FF1DAFF73
:100D40006F007BFFF6FF6F0077FFF7FF000EF86E76
:100D50000800F5502A0AD8A4B0EF86F0B2EF86F06A
:100D6000E5EF86F060000BF1D9FF60000FF1DAFFCC
:100D7000DE2A000EDD22600013F1D9FF600017F1BA
:100D8000DAFF6F007CFF46F0020EDE266F007CFF6C
:100D900047F0000EDD2260001BF1D9FF60001FF15B
:100DA000DAFF6F0078FFC6F06F0074FFC7F0C7BFAF
:100DB000DEEF86F0DCEF86F027EF87F0CA81C66DA4
:100DC000C71FD8B0C72B27EF87F060000BF1D9FF02
:100DD00060000FF1DAFF6F0078FF08F06F0074FF1A
:100DE00009F0C2EC9CF008C0C6F009C0C7F002EFE1
:100DF00087F060000BF1D9FF60000FF1DAFFDE2A07
:100E0000000EDD22D00E466EFF0E476E60000BF125
:100E1000D9FF60000FF1DAFF6F007BFFF6FF6F0074
:100E200077FFF7FF000EF86E0800F550486E496A2C
:100E30004650482647504922495009E10A0E485C6D
:100E4000D8A025EF87F027EF87F0F9EF86F0600054
:100E50000BF1D9FF60000FF1DAFF6F007BFFF6FFA7
:100E60006F0077FFF7FF000EF86E0800F5502E0AAE
:100E7000D8A43DEF87F03FEF87F0CEEF87F0000E6C
:100E80000001C96F000EC86F60000BF1D9FF600050
:100E90000FF1DAFFDE2A000EDD2260000BF1D9FF30
:100EA00060000FF1DAFF6F007BFFF6FF6F0077FF46
:100EB000F7FF000EF86E0800F5502A0AD8A463EF79
:100EC00087F065EF87F08CEF87F060000BF1D9FFBA
:100ED00060000FF1DAFFDE2A000EDD22600013F160
:100EE000D9FF600017F1DAFF6F007CFF46F0020EB9
:100EF000DE266F007CFF47F0000EDD2260001BF154
:100F0000D9FF60001FF1DAFF6F0078FFC8F06F00B3
:100F100074FFC9F0CEEF87F060000BF1D9FF6000DD
:100F20000FF1DAFF6F0078FF08F06F0074FF09F02F
:100F3000C2EC9CF008C0C8F009C0C9F0A9EF87F066
:100F400060000BF1D9FF60000FF1DAFFDE2A000E1E
:100F5000DD22D00E466EFF0E476E60000BF1D9FF0A
:100F600060000FF1DAFF6F007BFFF6FF6F0077FF85
:100F7000F7FF000EF86E0800F550486E496A4650BB
:100F8000482647504922495009E10A0E485CD8A03A
:100F9000CCEF87F0CEEF87F0A0EF87F060000BF189
:100FA000D9FF60000FF1DAFF6F007BFFF6FF6F00E3
:100FB00077FFF7FF000EF86E0800F550076E086A1D
:100FC0005DECADF007500001A86FA851D8B4EBEF6D
:100FD00087F0EDEF87F037EF88F060000BF1D9FF75
:100FE00060000FF1DAFF6F0078FF46F06F0074FFCA
:100FF00047F0010E4626000E472260001BF1F6FF67
:1010000060001FF1F7FF000EF86E0800F550076E44
:10101000086A5DECADF007500001A96FA951D8B482
:1010200014EF88F016EF88F037EF88F060000BF1CE
:10103000D9FF60000FF1DAFF6F0078FF46F06F0014
:1010400074FF47F0020E4626000E472260001BF197
:10105000F6FF60001FF1F7FF000EF86E0800F55074
:10106000076E086A5DECADF007500001AA6F6000E2
:101070000BF1D9FF60000FF1DAFF6F007BFFF6FF85
:101080006F0077FFF7FF000EF86E0800F550630A57
:10109000D8A44DEF88F04FEF88F07EEF88F0600025
:1010A0000BF1D9FF60000FF1DAFFDE2A000EDD221E
:1010B000600013F1D9FF600017F1DAFF6F007CFFC9
:1010C00046F0020EDE266F007CFF47F0000EDD22A8
:1010D00060001BF1D9FF60001FF1DAFFDF50AB6F3A
:1010E00040C00AF041C00BF0ABC00CF0D2ECA2F053
:1010F0000AC040F00BC041F055EF8BF060000BF1DF
:10110000D9FF60000FF1DAFF6F007BFFF6FF6F0081
:1011100077FFF7FF000EF86E0800F550640AD8B4A8
:1011200094EF88F096EF88F0AEEF88F060000BF156
:10113000D9FF60000FF1DAFF6F007BFFF6FF6F0051
:1011400077FFF7FF000EF86E0800F550690AD8A483
:10115000ACEF88F0AEEF88F0F8EF88F060000BF1AC
:10116000D9FF60000FF1DAFFDE2A000EDD226000F9
:1011700013F1D9FF600017F1DAFF6F007CFF46F032
:10118000020EDE266F007CFF47F0000EDD226000BD
:101190001BF1D9FF60001FF1DAFF6F0078FF92F0BA
:1011A0006F0074FF93F0000E93BFFF0E946F956F66
:1011B000966F976F986F996F40C01CF041C01DF0FB
:1011C00092C01EF093C01FF094C020F095C021F093
:1011D00096C022F097C023F098C024F099C025F063
:1011E00021EC95F01CC040F01DC041F055EF8BF094
:1011F000660EA819D8A4FFEF88F001EF89F054EF2C
:1012000089F060000BF1D9FF60000FF1DAFF6F0089
:101210007BFFF6FF6F0077FFF7FF000EF86E080008
:101220006F00D4FFABF060000BF1D9FF60000FF14D
:10123000DAFFDE2A000EDD22600013F1D9FF600024
:1012400017F1DAFF6F007CFF46F0040EDE266F0018
:101250007CFF47F0000EDD2260001BF1D9FF60002B
:101260001FF1DAFF6F0078FFA4F06F0078FFA5F0A0
:101270006F0078FFA6F06F0078FFA7F040C034F051
:1012800041C035F0A4C036F0A5C037F0A6C038F094
:10129000A7C039F0ABC03AF000EC80F034C040F0A9
:1012A00035C041F055EF8BF0A80E016E000E026EB6
:1012B000FB0E036EFF0E046E000E066E020E056E30
:1012C000F1ECA0F001500210D8A469EF89F06BEFA7
:1012D00089F0FEEF89F060000BF1D9FF60000FF19B
:1012E000DAFF6F0078FF46F06F0074FF47F0010EE1
:1012F0004626000E472260001BF1F6FF60001FF13A
:10130000F7FF000EF86E08006F00D4FFABF0BF0EC1
:10131000466EFF0E476E60000BF1D9FF60000FF1C3
:10132000DAFF6F007BFFF6FF6F0077FFF7FF000E1D
:10133000F86E0800F550486E496A465048264750F6
:101340004922495007E11A0E485CD8B0AAEF89F04B
:10135000ACEF89F0D0EF89F0600013F1D9FF6000A5
:1013600017F1DAFF6F007CFF46F0040EDE266F00F7
:101370007CFF47F0000EDD2260001BF1D9FF60000A
:101380001FF1DAFF6F0078FFA4F06F0078FFA5F07F
:101390006F0078FFA6F06F0078FFA7F0F2EF89F0FA
:1013A000600013F1D9FF600017F1DAFF6F007CFFD6
:1013B00046F0040EDE266F007CFF47F0000EDD22B3
:1013C00060001BF1D9FF60001FF1DAFF6F0078FFAA
:1013D000A4F06F0078FFA5F06F0078FFA6F06F0013
:1013E00078FFA7F0020E60000BF1D9FF60000FF14B
:1013F000DAFFDE26000EDD223EEF89F060000BF101
:10140000D9FF60000FF1DAFF6F007BFFF6FF6F007E
:1014100077FFF7FF000EF86E0800F550750AD8A4A4
:1014200014EF8AF016EF8AF062EF8AF060000BF199
:10143000D9FF60000FF1DAFFDE2A000EDD22600026
:1014400013F1D9FF600017F1DAFF6F007CFF46F05F
:10145000020EDE266F007CFF47F0000EDD226000EA
:101460001BF1D9FF60001FF1DAFF6F0078FF48F031
:101470006F0074FF49F048C09CF049C09DF0000126
:101480009E6B9F6BA06BA16BA26BA36B40C01CF00B
:1014900041C01DF09CC01EF09DC01FF09EC020F0FA
:1014A0009FC021F0A0C022F0A1C023F0A2C024F070
:1014B000A3C025F022EC9AF01CC040F01DC041F002
:1014C00055EF8BF060000BF1D9FF60000FF1DAFFF0
:1014D0006F007BFFF6FF6F0077FFF7FF000EF86EDF
:1014E0000800F550780AD8B478EF8AF07AEF8AF0DD
:1014F00092EF8AF060000BF1D9FF60000FF1DAFF84
:101500006F007BFFF6FF6F0077FFF7FF000EF86EAE
:101510000800F550580AD8A490EF8AF092EF8AF0AC
:10152000F2EF8AF060000BF1D9FF60000FF1DAFFF3
:101530006F007BFFF6FF6F0077FFF7FF000EF86E7E
:1015400008006F00D4FFABF060000BF1D9FF600022
:101550000FF1DAFFDE2A000EDD22600013F1D9FF61
:10156000600017F1DAFF6F007CFF46F0020EDE2606
:101570006F007CFF47F0000EDD2260001BF1D9FFF9
:1015800060001FF1DAFF6F0078FF48F06F0074FF12
:1015900049F048C09CF049C09DF000019E6B9F6BD4
:1015A000A06BA16BA26BA36B40C01CF041C01DF0EF
:1015B0009CC01EF09DC01FF09EC020F09FC021F077
:1015C000A0C022F0A1C023F0A2C024F0A3C025F047
:1015D000ABC026F094EC96F01CC040F01DC041F06A
:1015E00055EF8BF060000BF1D9FF60000FF1DAFFCF
:1015F0006F007BFFF6FF6F0077FFF7FF000EF86EBE
:101600000800F550250AD8A408EF8BF00AEF8BF0FC
:1016100023EF8BF060000BF1D9FF60000FF1DAFFD0
:10162000DE2A000EDD22000E026E250E016E40C085
:1016300003F041C004F03EECA3F0000E416E010E39
:10164000406E55EF8BF060000BF1D9FF60000FF199
:10165000DAFFDE2A000EDD22000E416E000E406E23
:1016600055EF8BF060000BF1D9FF60000FF1DAFF4E
:101670006F007BFFF6FF6F0077FFF7FF000EF86E3D
:101680000800F550016E026A40C003F041C004F04A
:101690003EECA3F060000BF1D9FF60000FF1DAFF20
:1016A000DE2A000EDD221DEF8BF012000450800BAD
:1016B0000D6E045004240F6E03AE61EF8BF063EFE8
:1016C0008BF064EF8BF00F800F50D8B46AEF8BF083
:1016D0006CEF8BF081EF8BF00F28D8A472EF8BF0BA
:1016E00074EF8BF07CEF8BF0000E016E000E026E3B
:1016F000000E036E000E046E038E000E046E89EF62
:101700008BF0000E016E000E026E000E036E000ED6
:10171000046E0850800B0E6E0D500E18D8B493EF67
:101720008BF095EF8BF096EF8BF00D8C0850082422
:101730000E6E07AE9EEF8BF0A0EF8BF0A1EF8BF05B
:101740000E800E50D8B4A7EF8BF0A9EF8BF0BEEF50
:101750008BF00E28D8A4AFEF8BF0B1EF8BF0B9EF80
:101760008BF0000E056E000E066E000E076E000E6A
:10177000086E078E000E086EC6EF8BF0000E056E29
:10178000000E066E000E076E000E086E0F500E5C07
:10179000D8B0CDEF8BF0CFEF8BF0F6EF8BF00DAC38
:1017A000D4EF8BF0D6EF8BF0D8EF8BF0800E0D1AC4
:1017B0000FC010F00EC00FF010C00EF001C010F0FE
:1017C00005C001F010C005F002C010F006C002F024
:1017D00010C006F003C010F007C003F010C007F0FF
:1017E00004C010F008C004F010C008F0000E106E25
:1017F0000F500EC009F00A6A095E000E0A5A0ABEAE
:101800000BEF8CF00A5009E11A0E095CD8A00BEF1F
:101810008CF00DEF8CF044EF8CF0015002100310AF
:101820000410D8A416EF8CF019EF8CF0010E1AEF0B
:101830008CF0000E106E000E016E000E026E000E97
:10184000036E000E046E0EC00FF04DEF8CF010A072
:101850002CEF8CF02EEF8CF034EF8CF0D890103011
:101860000109106E36EF8CF0D890103201A03BEFDA
:101870008CF03DEF8CF03EEF8CF0108E043404328F
:101880000332023201320F2A0E500F5CD8A04BEF08
:101890008CF04DEF8CF027EF8CF00DBC52EF8CF0FC
:1018A00054EF8CF094EF8CF00F50D8A45AEF8CF0DA
:1018B0005CEF8CF066EF8CF0000E016E000E026E95
:1018C000000E036E000E046EB5EF8DF0055001267C
:1018D00006500222075003220850042204A073EF8E
:1018E0008CF075EF8CF021EF8DF010A07AEF8CF07A
:1018F0007CEF8CF082EF8CF0D89010300109106EE4
:1019000084EF8CF0D890103201A089EF8CF08BEF2F
:101910008CF08CEF8CF0108E0434043203320232DF
:1019200001320F2A21EF8DF00550015C065002585C
:10193000075003580450800A096E0850800A09585D
:10194000D8B0A5EF8CF0A7EF8CF0D2EF8CF001505F
:10195000055C096E025006580A6E035007580B6E5C
:10196000045008580C6EFF0E0924016EFF0E0A2069
:10197000026EFF0E0B20036EFF0E0C20046E800E15
:101980000D1A106C1050D8A4C8EF8CF0CAEF8CF070
:10199000DAEF8CF0010E0126000E0222032204224F
:1019A000DAEF8CF00550015E0650025A0750035AD8
:1019B0000850045A0150021003100410D8A4E3EF99
:1019C0008CF0E5EF8CF01AEF8DF01050D8A4EBEF0F
:1019D0008CF0EDEF8CF01AEF8DF0000E016E000E22
:1019E000026E000E036E000E046EB5EF8DF0D890FF
:1019F000013602360336043610AE01EF8DF003EFE8
:101A00008DF004EF8DF0018010A009EF8DF00BEF49
:101A10008DF00FEF8DF0D880103611EF8DF0D8904B
:101A200010360F50D8B417EF8DF019EF8DF01AEF74
:101A30008DF00F0603AE1FEF8DF021EF8DF0F7EF65
:101A40008CF0000E0E6E10AE28EF8DF02AEF8DF0A8
:101A500042EF8DF010C009F07F0E0916D8B433EFB5
:101A60008DF035EF8DF039EF8DF0010E0E6E42EFF7
:101A70008DF001A03EEF8DF040EF8DF042EF8DF044
:101A800035EF8DF00E50D8B448EF8DF04AEF8DF061
:101A900075EF8DF0010E0126000E022203220422B2
:101AA00004A055EF8DF057EF8DF075EF8DF001C06C
:101AB00009F002C00AF003C00BF004C00CF00C34B3
:101AC0000C320B320A32093209C001F00AC002F0AE
:101AD0000BC003F00CC004F00F28D8B472EF8DF0E7
:101AE00074EF8DF075EF8DF00F2A0F28D8B47BEFCF
:101AF0008DF07DEF8DF085EF8DF00F50D8A483EF42
:101B00008DF085EF8DF097EF8DF0000E016E000ED9
:101B1000026E000E036E000E046E0F50D8A493EFF9
:101B20008DF095EF8DF097EF8DF0000E0D6E0FA0FC
:101B30009CEF8DF09EEF8DF0A1EF8DF0038EA2EF64
:101B40008DF0039ED8900F30046E0DAEAAEF8DF08D
:101B5000ACEF8DF0ADEF8DF0048E01C001F002C04E
:101B600002F003C003F004C004F012001250800B16
:101B70001B6E12501224216E11AEC1EF8DF0C3EF17
:101B80008DF0C4EF8DF021802150D8B4CAEF8DF0D4
:101B9000CCEF8DF0DFEF8DF02128D8A4D2EF8DF0BF
:101BA000D4EF8DF0DCEF8DF0000E0F6E000E106E96
:101BB000000E116E000E126E118EE7EF8DF0000E0A
:101BC0000F6E000E106E000E116E000E126E16508B
:101BD000800B1B1A16501624206E15AEF2EF8DF0F6
:101BE000F4EF8DF0F5EF8DF020802050D8B4FBEFAE
:101BF0008DF0FDEF8DF010EF8EF02028D8A403EFCC
:101C00008EF005EF8EF00DEF8EF0000E136E000ECD
:101C1000146E000E156E000E166E158E18EF8EF0F7
:101C2000000E136E000E146E000E156E000E166E72
:101C30002050D8B41EEF8EF020EF8EF028EF8EF0FB
:101C40002150D8A426EF8EF028EF8EF032EF8EF0E0
:101C5000000E0F6E000E106E000E116E000E126E52
:101C6000DCEF8FF015500F026F00CCFF26F06F00F5
:101C7000D0FF27F026501C6E1D6A1E6A1F6A27506F
:101C8000226E236A246A256A145010026F00CCFF6A
:101C900026F06F00D0FF27F026501C26000E1D22D4
:101CA0001E221F2227502226000E23222422252214
:101CB000135011026F00CCFF26F06F00D0FF27F009
:101CC00026501C26000E1D221E221F2227502226CF
:101CD000000E2322242225221EC01FF01DC01EF04C
:101CE0001CC01DF01C6A135010026F00CCFF26F0C0
:101CF0006F00D0FF27F026501C2627501D22000E13
:101D00001E22000E1F2214500F026F00CCFF26F07F
:101D10006F00D0FF27F026501C2627501D22000EF2
:101D20001E22000E1F221EC01FF01DC01EF01CC070
:101D30001DF01C6A13500F026F00CCFF26F06F00DD
:101D4000D0FF27F026501C2627501D22000E1E22F1
:101D5000000E1F22155010026F00CCFF26F06F00FE
:101D6000D0FF27F02650222627502322000E2422BF
:101D7000000E2522145011026F00CCFF26F06F00D8
:101D8000D0FF27F02650222627502322000E24229F
:101D9000000E2522155011026F00CCFF26F06F00B7
:101DA000D0FF27F02650176E2750186E196A1A6A4E
:101DB00019C01AF018C019F017C018F0176A175098
:101DC000222618502322195024221A5025221CC0E2
:101DD00017F01DC018F01EC019F01FC01AF0190E20
:101DE000F7EF8EF0D8901A32193218321732E82EE7
:101DF000F2EF8EF017502226185023221950242279
:101E00001A5025221EC01FF01DC01EF01CC01DF060
:101E10001C6A205021C017F0186A1726000E1822DD
:101E2000820E1724266EFF0E1820276E2DEF8FF0DE
:101E3000D89022362336243625361FAE22EF8FF077
:101E400024EF8FF025EF8FF02280D8901C361D36BE
:101E50001E361F362606D8A0270624AE32EF8FF096
:101E600034EF8FF018EF8FF0000E206E1FAE3BEFB7
:101E70008FF03DEF8FF061EF8FF0FF0E1C14176EA7
:101E8000FF0E1D14186EFF0E1E14196E7F0E1F1408
:101E90001A6E1750181019101A10D8B452EF8FF08C
:101EA00054EF8FF058EF8FF0010E206E61EF8FF03E
:101EB00022A05DEF8FF05FEF8FF061EF8FF054EFB6
:101EC0008FF02050D8B467EF8FF069EF8FF08DEF6F
:101ED0008FF0010E2226000E23222422252225A087
:101EE00074EF8FF076EF8FF08DEF8FF022C017F048
:101EF00023C018F024C019F025C01AF01A341A3281
:101F000019321832173217C022F018C023F019C046
:101F100024F01AC025F0264A272A27BE98EF8FF012
:101F2000275008E12628D8A098EF8FF09AEF8FF07D
:101F3000A4EF8FF0000E226E000E236E800E246E32
:101F40007F0E256ED2EF8FF027BEB1EF8FF02750B6
:101F500006E12604D8B0AFEF8FF0B1EF8FF0BDEF00
:101F60008FF0000E226E000E236E000E246E000E07
:101F7000256E000E1B6ED2EF8FF026C021F0FF0EF3
:101F80002216FF0E23167F0E2416000E251621A002
:101F9000CCEF8FF0CEEF8FF0CFEF8FF0248ED89074
:101FA0002130256E1B50251222C00FF023C010F0E7
:101FB00024C011F025C012F012000450800B116EE5
:101FC00004500424186E03AEE8EF8FF0EAEF8FF0B0
:101FD000EBEF8FF018801850D8B4F1EF8FF0F3EFDB
:101FE0008FF008EF90F01828D8A4F9EF8FF0FBEFEE
:101FF0008FF003EF90F0000E016E000E026E000EE7
:10200000036E000E046E038E000E046E10EF90F04F
:10201000000E016E000E026E000E036E000E046EC6
:102020000850800B111A08500824196E07AE1BEFD8
:1020300090F01DEF90F01EEF90F019801950D8B479
:1020400024EF90F026EF90F03BEF90F01928D8A401
:102050002CEF90F02EEF90F036EF90F0000E056E22
:10206000000E066E000E076E000E086E078E000E44
:10207000086E43EF90F0000E056E000E066E000E27
:10208000076E000E086E0550061007100810D8A441
:102090004CEF90F04EEF90F066EF90F0000E016E76
:1020A000000E026E000E036E000E046E800E031210
:1020B0007F0E04121150041201C001F002C002F0A0
:1020C00003C003F004C004F0A9EF91F01850D8A4A5
:1020D0006CEF90F06EEF90F078EF90F0000E016EE4
:1020E000000E026E000E036E000E046EA9EF91F05A
:1020F000195018C009F00A6A095E000E0A5A7F0ECC
:102100000924126E000E0A20136E01C00DF002C0E9
:102110000EF003C00FF004C010F0000E016E000EB0
:10212000026E000E036E000E046E000E146E000EA2
:10213000156E000E166E000E176E000E196ED9EF9A
:1021400090F01950D8B4A7EF90F0A9EF90F0C0EF3D
:1021500090F0D8900D360E360F361036D8900136E6
:1021600002360336043617AEB8EF90F0BAEF90F0AF
:10217000BBEF90F00180D89014361536163617361E
:1021800005500D5C06500E5807500F580850105857
:10219000D8A0CDEF90F0CFEF90F0D8EF90F0178C63
:1021A00005500D5E06500E5A07500F5A0850105A2F
:1021B000192A190E1964DFEF90F0E1EF90F0A1EF0A
:1021C00090F00D500E100F101010D8B4EAEF90F0F0
:1021D000ECEF90F004EF91F0148004EF91F0D890C0
:1021E000013602360336043617AEF9EF90F0FBEFF6
:1021F00090F0FCEF90F00180D8901436153616362A
:1022000017361206D8A0130603AE09EF91F00BEFB4
:1022100091F0EFEF90F0000E196E17AE12EF91F003
:1022200014EF91F038EF91F0FF0E1414096EFF0EC9
:1022300015140A6EFF0E16140B6E7F0E17140C6E1B
:1022400009500A100B100C10D8B429EF91F02BEFA5
:1022500091F02FEF91F0010E196E38EF91F001A07F
:1022600034EF91F036EF91F038EF91F02BEF91F0E1
:102270001950D8B43EEF91F040EF91F064EF91F037
:10228000010E0126000E02220322042204A04BEFBD
:1022900091F04DEF91F064EF91F001C009F002C0B0
:1022A0000AF003C00BF004C00CF00C340C320B32FB
:1022B0000A32093209C001F00AC002F00BC003F073
:1022C0000CC004F0124A132A13BE6FEF91F01350A2
:1022D00008E11228D8A06FEF91F071EF91F07CEF38
:1022E00091F0000E136E1268000E016E000E026E69
:1022F000000E036E000E046E13BE89EF91F01350B2
:1023000006E11204D8B087EF91F089EF91F097EFD2
:1023100091F0000E136E000E126E000E016E000E94
:10232000026E000E036E000E046E000E116E12C0DF
:1023300018F018A09EEF91F0A0EF91F0A3EF91F0AC
:10234000038EA4EF91F0039ED8901830046E5AEFDC
:1023500090F01200600E3901D96F000EDB6F000E95
:10236000DD6F080EDF6F000EDE6F7A0E0001BF6FAB
:10237000C10EBE6F810EE82EFED7BE2FFCD7BF2F39
:10238000FAD700D0FDECA7F0C296BA96000E000175
:10239000DE6F030EDF6F000EF16F000EF06FF15174
:1023A00009E1800EF05DD8A0D8EF91F0DAEF91F05E
:1023B000DCEF91F0F1EF91F0000EF025D96E020EF6
:1023C000F121DA6E000EDF6EF04BF12BF15109E1D5
:1023D000800EF05DD8A0EFEF91F0F1EF91F0DCEF1F
:1023E00091F0000EF16F000EF06FF15109E1500E07
:1023F000F05DD8A0FEEF91F000EF92F002EF92F0C6
:1024000017EF92F0A00EF025D96E020EF121DA6ED0
:10241000000EDF6EF04BF12BF15109E1500EF05D33
:10242000D8A015EF92F017EF92F002EF92F039EC8E
:10243000ADF0290E0001BF6F960EBE6F7F0EE82E25
:10244000FED7BE2FFCD7BF2FFAD7F1ECAFF0660E48
:10245000076EFF0E086EF3ECABF0000E0001F16F9B
:10246000000EF06FF15109E1090EF05DD8A03BEFCD
:1024700092F03DEF92F03FEF92F05EEF92F0D89045
:10248000F035D96EF135DA6EC80ED926010EDA2292
:102490006F0078FF07F06F0074FF08F0F3ECABF00B
:1024A0000001F04BF12BF15109E1090EF05DD8A0CC
:1024B0005CEF92F05EEF92F03FEF92F0F1ECAFF054
:1024C000950E076EFF0E086EF3ECABF0C4ECB0F0A7
:1024D000D40E076EFD0E086EF3ECABF0E9EC97F04E
:1024E000F1ECAFF0200E0001F66F000EFF6F100E42
:1024F000FE6FA00EAC6F020EAD6F890EAE6FFE0EBA
:10250000AF6FF6C0B0F0B16BF6C0B2F0B36BC3EC16
:10251000ACF0A00E016E020E026E28ECAAF03D0196
:102520007589F1ECAFF0FA0E076EFD0E086EF3EC54
:10253000ABF03D01738F33EC9EF0010EFDECA8F083
:10254000010E1EECACF0020EFDECA8F0540E076E6E
:10255000FE0E086EF3ECABF0550E1F6EFF0E206EF4
:102560003BECA9F0000E256E020E246ED7ECA4F011
:10257000090E0001BF6F1E0EBE6FE40EE82EFED7DF
:10258000BE2FFCD7BF2FFAD700F0330E1F6EFF0E01
:10259000206E3BECA9F0020E1EECACF01A0E076E9A
:1025A000FE0E086EF3ECABF049ECAEF0A70E076E32
:1025B000FD0E086EF3ECABF09FECB0F0EA0E076E88
:1025C000FE0E086EF3ECABF06EECA1F0000E000115
:1025D000F16F000EF06F000E216E000E206E010EE6
:1025E0006AEC93F0010EFDECA8F0020EFDECA8F0F1
:1025F000220E1F6EFF0E206E3BECA9F0BD0E076E83
:10260000FE0E086EF3ECABF09FECB0F0BA86BC0E99
:10261000286E010E296E61ECA2F028C0C0F029C01E
:10262000C1F02AC0C2F02BC0C3F0BA96DEC0ACF035
:10263000DFC0ADF0380E0001AE6FFE0EAF6FF0C020
:10264000B0F0F1C0B1F0C0C0B2F0C1C0B3F0C2C0D0
:10265000B4F0C3C0B5F0000EB76FB00EB66FC3ECE8
:10266000ACF0DEC001F0DFC002F028ECAAF0A00E52
:102670000001AC6F020EAD6FDD0EAE6FFF0EAF6FDF
:10268000C0C0B0F0C1C0B1F0C2C0B2F0C3C0B3F0BE
:10269000C3ECACF00A0E256EA00E266E020E276E5D
:1026A000010E2EECB1F0000E216E010E206E000E18
:1026B000236E0F0E226E000E246E25ECA7F0BB7A5F
:1026C0000001F04BF12B020E1EECACF004EF93F086
:1026D00057EF00F0266E400EFDECA8F00D0E236EB5
:1026E0002D0E226ED80EE82EFED7222EFCD7232EDA
:1026F000FAD72604D8A47FEF93F081EF93F093EFFD
:1027000093F0000E026E000E016E000E046E070EB6
:10271000036E61ECB0F0260E0124076EFC0E022061
:10272000086EF3ECABF0020E2618D8A49AEF93F0E3
:102730009CEF93F0AEEF93F0000E026E000E016E70
:10274000000E046E070E036E61ECB0F0EE0E012475
:10275000076EFB0E0220086EF3ECABF0030E26189A
:10276000D8A4B5EF93F0B7EF93F0C9EF93F0000E54
:10277000026E000E016E000E046E070E036E61EC19
:10278000B0F0EE0E0124076EFB0E0220086EF3EC93
:10279000ABF0F1ECAFF0000E256E010E246E000ED2
:1027A000286E000E276E27502810D8B4DAEF93F069
:1027B000DCEF93F0D5EF94F0070E2714226E000E95
:1027C0002814236E22502310D8A4E9EF93F0EBEFE6
:1027D00093F0D5EF94F02604D8A4F1EF93F0F3EF43
:1027E00093F005EF94F024C001F025C002F0000E34
:1027F000046E070E036E61ECB0F0260E0124076E26
:10280000FC0E0220086EF3ECABF0020E2618D8A4E2
:102810000CEF94F00EEF94F020EF94F024C001F050
:1028200025C002F0000E046E070E036E61ECB0F0DE
:10283000EE0E0124076EFB0E0220086EF3ECABF0E7
:10284000030E2618D8A427EF94F029EF94F03BEF5D
:1028500094F024C001F025C002F0000E046E070EB3
:10286000036E61ECB0F0EE0E0124076EFB0E022049
:10287000086EF3ECABF0244A252AF1ECAFF0D5EF6B
:1028800094F0270E2724F66EFB0E2820F76EF86AC8
:10289000000EF8220800F550BFECA8F0200421102B
:1028A000D8A455EF94F057EF94F0EEEF94F0270E84
:1028B0002724F66EFB0E2820F76EF86A000EF82229
:1028C0000800F550A3ECADF0EEEF94F0E70E2724EE
:1028D000F66EFA0E2820F76EF86A000EF82208004D
:1028E000F550BFECA8F020042110D8A47AEF94F0A2
:1028F0007CEF94F0EEEF94F0E70E2724F66EFA0EDC
:102900002820F76EF86A000EF8220800F550A3ECB4
:10291000ADF0EEEF94F0A70E2724F66EFA0E282005
:10292000F76EF86A000EF8220800F550BFECA8F028
:1029300020042110D8A49FEF94F0A1EF94F0EEEFC3
:1029400094F0A70E2724F66EFA0E2820F76EF86A88
:10295000000EF8220800F550A3ECADF0EEEF94F075
:10296000270E2724F66EFB0E2820F76EF86A000E5D
:10297000F8220800F550BFECA8F020042110D8A4DC
:10298000C4EF94F0C6EF94F0EEEF94F0270E2724F6
:10299000F66EFB0E2820F76EF86A000EF82208008B
:1029A000F550A3ECADF0EEEF94F02650226E236AC2
:1029B0002350000AD8B4DFEF94F0B0EF94F0225027
:1029C000010AD8B441EF94F0030AD8B466EF94F04A
:1029D000010AD8B48BEF94F0B0EF94F0030E236E9D
:1029E000080E226E770EE82EFED7222EFCD7232E5D
:1029F000FAD700F020042110D8A401EF95F003EFDE
:102A000095F005EF95F0F1ECAFF0274A282A285011
:102A100009E1400E275CD8A010EF95F012EF95F079
:102A2000D3EF93F0800EFDECA8F00D0E236E2D0E6B
:102A3000226ED80EE82EFED7222EFCD7232EFAD7F0
:102A400012001EC036F01FC037F020C038F021C081
:102A500039F022C03AF023C03BF024C03CF025C03E
:102A60003DF03DBE36EF95F039EF95F0010E3AEFAF
:102A700095F0000E346E356A34503510D8B443EFFB
:102A800095F045EF95F055EF95F03D1E3C1E3B1E31
:102A90003A1E391E381E371E366C000E3722382279
:102AA00039223A223B223C223D220001C9BF5BEF82
:102AB00095F05DEF95F05EEF95F0CA93C9BF6BEFAF
:102AC00095F0C95106E1C805D8B069EF95F06BEFF4
:102AD00095F071EF95F0000E316E010E306E75EFCE
:102AE00095F0C8C030F0C9C031F0C6C032F0C7C0E0
:102AF00033F034503510D8A480EF95F082EF95F084
:102B000089EF95F0CAA587EF95F089EF95F08CEFE6
:102B100095F03206D8A03306000E3F6E4F0E3E6E83
:102B2000000E0101BB6F11EF96F03E06D8A03F06E4
:102B30006C0E3E24D96E010E3F20DA6E36C001F0D5
:102B400037C002F038C003F039C004F03AC005F0D5
:102B50003BC006F03CC007F03DC008F00A0E096E0D
:102B6000000E0A6E000E0B6E000E0C6E000E0D6E47
:102B7000000E0E6E000E0F6E000E106E81EC9DF0BA
:102B800001C026F002C027F003C028F004C029F0DD
:102B900005C02AF006C02BF007C02CF008C02DF0AD
:102BA00026C013F028C014F00AECAEF01350300F1A
:102BB000DF6E3006D8A031063206D8A0330636C004
:102BC00001F037C002F038C003F039C004F03AC059
:102BD00005F03BC006F03CC007F03DC008F00A0E0F
:102BE000096E000E0A6E000E0B6E000E0C6E000ECB
:102BF0000D6E000E0E6E000E0F6E000E106EFEECCF
:102C00009BF001C036F002C037F003C038F004C0BA
:102C100039F005C03AF006C03BF007C03CF008C0F0
:102C20003DF03FBE1CEF96F03F5008E13E04D8A0B7
:102C30001CEF96F01EEF96F04FEF96F036503710DF
:102C4000381039103A103B103C103D10D8A42BEF2F
:102C500096F02DEF96F095EF95F031BE3AEF96F0A5
:102C6000315006E13004D8B038EF96F03AEF96F0E4
:102C700095EF95F033BE45EF96F0335008E13204FE
:102C8000D8A045EF96F047EF96F04FEF96F0000191
:102C9000CAB34DEF96F04FEF96F095EF95F03450A4
:102CA0003510D8A456EF96F058EF96F060EF96F0F6
:102CB0000001CAA55EEF96F060EF96F07FEF96F008
:102CC0003E06D8A03F0634503510D8A46AEF96F0DF
:102CD0006CEF96F072EF96F0000E2F6E2B0E2E6EAC
:102CE00076EF96F0000E2F6E2D0E2E6E6C0E3E249B
:102CF000D96E010E3F20DA6E6000BBF0DFFF1CC012
:102D000011F01DC012F06C0E3E24136E010E3F2018
:102D1000146E32C015F033C016F012ECA4F011C0DE
:102D20001CF012C01DF012000001C9BF9AEF96F00E
:102D30009CEF96F09DEF96F0CA93C9BFAAEF96F06C
:102D4000C95106E1C805D8B0A8EF96F0AAEF96F0F1
:102D5000B0EF96F0000E306E010E2F6EB4EF96F0CD
:102D6000C8C02FF0C9C030F0C6C031F0C7C032F0C3
:102D7000CAA9BDEF96F0BFEF96F0C3EF96F0FE0E36
:102D80003126FF0E32221EC033F01FC034F020C0A7
:102D900035F021C036F022C037F023C038F024C00F
:102DA00039F025C03AF0000E3C6E4F0E3B6E000E1F
:102DB0000101BB6F76EF97F03B06D8A03C060F0EE3
:102DC00033143D6E3E6A3EBEEFEF96F03E5009E191
:102DD0000A0E3D5CD8A0EFEF96F0F1EF96F0F9EF18
:102DE00096F0570E3D243D6E000E3E203E6EFFEFE6
:102DF00096F0300E3D243D6E000E3E203E6EBF0E1E
:102E0000276EFF0E286E2650296E2A6A2750292623
:102E100028502A222A5007E11A0E295CD8B013EF55
:102E200097F015EF97F038EF97F09F0E276EFF0E93
:102E3000286E200E3D10296E000E3E102A6E27507F
:102E4000292628502A222A5007E11A0E295CD8B0D8
:102E50002CEF97F02EEF97F038EF97F03DC007F08A
:102E60003EC008F0C6ECADF007C03DF008C03EF033
:102E70006C0E3B24D96E010E3C20DA6E6000F7F038
:102E8000DFFF2F06D8A030063106D8A0320633C0A7
:102E900027F034C028F035C029F036C02AF037C0FA
:102EA0002BF038C02CF039C02DF03AC02EF0050EB2
:102EB00063EF97F0D8902E322D322C322B322A32FB
:102EC000293228322732E82E5AEF97F027C033F004
:102ED00028C034F029C035F02AC036F02BC037F0B6
:102EE0002CC038F02DC039F02EC03AF03CBE82EF35
:102EF00097F03C5009E1020E3B5CD8A082EF97F0BE
:102F000084EF97F0B5EF97F033503410351036104A
:102F10003710381039103A10D8A491EF97F093EF8A
:102F200097F0DCEF96F030BEA0EF97F0305006E15E
:102F30002F04D8B09EEF97F0A0EF97F0DCEF96F05B
:102F400032BEABEF97F0325008E13104D8A0ABEFBE
:102F500097F0ADEF97F0B5EF97F00001CAB3B3EF7C
:102F600097F0B5EF97F0DCEF96F00001CAA9BBEF40
:102F700097F0BDEF97F0D4EF97F03B06D8A03C0652
:102F80006C0E3B24D96E010E3C20DA6E60009BF083
:102F9000DFFF3B06D8A03C066C0E3B24D96E010E29
:102FA0003C20DA6E300EDF6E1CC011F01DC012F036
:102FB0006C0E3B24136E010E3C20146E31C015F0D4
:102FC00032C016F012ECA4F011C01CF012C01DF0BB
:102FD0001200000E0001DE6F030EDF6F60007BF356
:102FE000D9FF60007FF3DAFF000EDF6E3D017599B7
:102FF000738F000E0001BD6F020EBC6FBCC001F0EC
:10300000BDC002F049ECAFF00009D8B40AEF98F067
:103010000CEF98F0FEEF98F00001BD35BD31B86FB0
:10302000BC31EC6FB8C0EDF0DEC0ACF0DFC0ADF08D
:10303000790EAE6FFD0EAF6FBCC0B0F0BDC0B1F089
:10304000ECC0B2F0EDC0B3F0C3ECACF0A7EF98F079
:10305000DEC00FF0DFC010F0A30E116EFE0E126E78
:10306000DAECAFF00FC0DEF010C0DFF0F6EF98F052
:10307000A00E016E020E026E440E036EFF0E046E71
:103080002AECAEF0DEC001F0DFC002F085ECAEF05D
:1030900001C0BAF002C0BBF00001BA51DE25056ED6
:1030A000BB51DF21066EA00E076E020E086E03EC08
:1030B000ABF0F6EF98F0DEC00FF0DFC010F0100EAE
:1030C000116EFF0E126EDAECAFF00FC0DEF010C022
:1030D000DFF0F6EF98F0DEC00FF0DFC010F0FD0E6D
:1030E000116EFE0E126EDAECAFF0F6EF98F0DEC065
:1030F0000FF0DFC010F0A40E116EFF0E126EDAECAE
:10310000AFF0F6EF98F0DEC00FF0DFC010F0760EF3
:10311000116EFF0E126EDAECAFF0F6EF98F0DEC033
:103120000FF0DFC010F0C90E116EFF0E126EDAEC58
:10313000AFF0F6EF98F0DEC00FF0DFC010F0BD0E7C
:10314000116EFF0E126EDAECAFF0F6EF98F0ECC0F5
:10315000B8F0EDC0B9F00001B951000AD8B4B3EF2E
:1031600098F09BEF98F0B851200AD8B428EF98F067
:10317000010AD8B428EF98F0030AD8B428EF98F0E1
:10318000010AD8B428EF98F0040AD8B428EF98F0D0
:103190000F0AD8B438EF98F0010AD8B438EF98F095
:1031A000030AD8B438EF98F01D0AD8B45BEF98F052
:1031B0000F0AD8B46BEF98F0010AD8B46BEF98F00F
:1031C000030AD8B46BEF98F0010AD8B46BEF98F00B
:1031D000070AD8B477EF98F06B0AD8B483EF98F069
:1031E0003F0AD8B48FEF98F09BEF98F0DEC001F063
:1031F000DFC002F028ECAAF0F1ECAFF0020E000103
:10320000BC25BC6F000EBD21BD6FBDBF11EF99F095
:10321000BD5109E1FC0EBC5DD8A011EF99F013EF90
:1032200099F0FEEF97F03D01739F7589F1ECAFF0D7
:1032300012004AC12AF04BC12BF04CC12CF04DC1F9
:103240002DF01AC02AF01BC02BF01CC02CF01DC0A2
:103250002DF0810E1E6EFF0E1F6E2AC020F02BC0B7
:1032600021F02CC022F02DC023F0180E3DEF99F074
:10327000D8902332223221322032E82E38EF99F0D2
:1032800020501E24286E000E1F20296E29BE52EFEA
:1032900099F0295009E1170E285CD8A052EF99F057
:1032A00054EF99F05EEF99F01AC01AF01BC01BF0B2
:1032B0001CC01CF01DC01DF021EF9AF029BE63EF69
:1032C00099F065EF99F0D5EF99F028C01EF0FF0E48
:1032D0001F6EFF0E206E7F0E216E000E226E1E6688
:1032E00074EF99F07CEF99F02234223221322032AF
:1032F0001F321E2E6FEF99F01FC024F020C025F062
:1033000021C026F022C027F024502A141E6E25501A
:103310002B141F6E26502C14206E27502D14216E56
:103320001E501F1020102110D8A499EF99F09BEF88
:1033300099F09DEF99F054EF99F02AC01EF02BC040
:103340001FF02CC020F02DC021F0200EADEF99F021
:10335000D890213220321F321E32E82EA8EF99F089
:103360001E501F1020102110D8B4B9EF99F0BBEFF8
:1033700099F0C3EF99F024502A2625502B2226508D
:103380002C2227502D22241C1E6E251C1F6E261C4D
:10339000206E271C216E1E502A161F502B162050FF
:1033A0002C1621502D1619EF9AF02AC01EF02BC0B2
:1033B0001FF02CC020F02DC021F0200EE5EF99F079
:1033C000D890213220321F321E32E82EE0EF99F0E1
:1033D0001E501F1020102110D8A4F1EF99F0F3EF28
:1033E00099F0FDEF99F0000E2A6E000E2B6E000E84
:1033F0002C6E000E2D6E19EF9AF0D8902A341E6EA6
:103400002B341F6E2C34206E2D34216E1E501F1055
:1034100020102110D8B40FEF9AF011EF9AF019EFA5
:103420009AF0000E2A6E000E2B6E800E2C6EBF0ED0
:103430002D6E2AC01AF02BC01BF02CC01CF02DC022
:103440001DF012000001C9BF28EF9AF02AEF9AF090
:103450002BEF9AF0CA93C9BF38EF9AF0C95106E131
:10346000C805D8B036EF9AF038EF9AF03EEF9AF0F0
:10347000000E2F6E010E2E6E42EF9AF0C8C02EF095
:10348000C9C02FF0C6C030F0C7C031F01EC032F046
:103490001FC033F020C034F021C035F022C036F018
:1034A00023C037F024C038F025C039F0000E3B6E41
:1034B0004F0E3A6E000E0101BB6FD5EF9AF03A063F
:1034C000D8A03B066C0E3A24D96E010E3B20DA6E72
:1034D00032C001F033C002F034C003F035C004F054
:1034E00036C005F037C006F038C007F039C008F024
:1034F0000A0E096E000E0A6E000E0B6E000E0C6EA8
:10350000000E0D6E000E0E6E000E0F6E000E106E91
:10351000AAECA3F001C026F002C027F003C028F0F7
:1035200004C029F005C02AF006C02BF007C02CF01B
:1035300008C02DF02650300FDF6E2E06D8A02F06C3
:103540003006D8A0310632C001F033C002F034C0DA
:1035500003F035C004F036C005F037C006F038C0BF
:1035600007F039C008F00A0E096E000E0A6E000E50
:103570000B6E000E0C6E000E0D6E000E0E6E000E29
:103580000F6E000E106EE9ECA1F001C032F002C027
:1035900033F003C034F004C035F005C036F006C087
:1035A00037F007C038F008C039F03A503B10D8B4B3
:1035B000DCEF9AF0DEEF9AF00FEF9BF03250331011
:1035C000341035103610371038103910D8A4EBEFFE
:1035D0009AF0EDEF9AF05FEF9AF02FBEFAEF9AF0C3
:1035E0002F5006E12E04D8B0F8EF9AF0FAEF9AF0D7
:1035F0005FEF9AF031BE05EF9BF0315008E13004E7
:10360000D8A005EF9BF007EF9BF00FEF9BF00001B8
:10361000CAB30DEF9BF00FEF9BF05FEF9AF01CC069
:1036200011F01DC012F06C0E3A24136E010E3B20F7
:10363000146E30C015F031C016F012ECA4F011C0B9
:103640001CF012C01DF01200096E0950D8B42BEF07
:103650009BF02DEF9BF04FEF9BF004BE34EF9BF0FF
:1036600032EF9BF04FEF9BF001C005F002C006F077
:1036700003C007F004C008F0051E061E071E081E42
:10368000052A000E06220722082205C00BF006C0FC
:103690000CF007C00DF008C00EF057EF9BF001C012
:1036A0000BF002C00CF003C00DF004C00EF001508E
:1036B000021003100410D8A460EF9BF062EF9BF09F
:1036C0006CEF9BF0000E016E000E026E000E036E9A
:1036D000000E046EFDEF9BF0960E0A6E76EF9BF0E7
:1036E0000A2AD8900E320D320C320B32000E0B1417
:1036F000056E000E0C14066E000E0D14076EFE0E05
:103700000E14086E0550061007100810D8A48BEF91
:103710009BF08DEF9BF070EF9BF09BEF9BF00A2AE4
:10372000010E0B26000E0C220D220E22D8900E3216
:103730000D320C320B32000E0B14056E000E0C1401
:10374000066E000E0D14076EFF0E0E14086E055067
:10375000061007100810D8A4B0EF9BF0B2EF9BF052
:103760008FEF9BF0BAEF9BF00A06D8900B360C3621
:103770000D360E360DBEBFEF9BF0C1EF9BF0C9EFCB
:103780009BF0020E0A60C7EF9BF0C9EF9BF0B4EF0D
:103790009BF00AB0CEEF9BF0D0EF9BF0D1EF9BF007
:1037A0000D9ED8900A320AC005F0066A076A086AB8
:1037B00005C008F0076A066A056A05500B12065034
:1037C0000C1207500D1208500E120950D8B4EBEF2E
:1037D0009BF0EDEF9BF0F5EF9BF004BEF4EF9BF058
:1037E000F2EF9BF0F5EF9BF00E8E0BC001F00CC0DA
:1037F00002F00DC003F00EC004F01200000E126EB5
:1038000010BE07EF9CF005EF9CF019EF9CF0101E26
:103810000F1E0E1E0D1E0C1E0B1E0A1E096C000E26
:103820000A220B220C220D220E220F221022010E40
:10383000126E08BE20EF9CF01EEF9CF032EF9CF061
:10384000081E071E061E051E041E031E021E016C16
:10385000000E022203220422052206220722082249
:10386000010E121A20EE13F0070EDE6AE806FDE2E2
:1038700009500A100B100C100D100E100F10101024
:10388000D8B445EF9CF047EF9CF099EF9CF0010E07
:10389000116E55EF9CF0D89009360A360B360C366F
:1038A0000D360E360F361036112A10AE5AEF9CF038
:1038B0005CEF9CF04BEF9CF0D89013361436153625
:1038C00016361736183619361A360950015C0A5062
:1038D00002580B5003580C5004580D5005580E5008
:1038E00006580F50075810500858D8A07AEF9CF08F
:1038F0007CEF9CF08DEF9CF00950015E0A50025A5B
:103900000B50035A0C50045A0D50055A0E50065ACB
:103910000F50075A1050085A1380D89010320F32A7
:103920000E320D320C320B320A320932112E5CEF9C
:103930009CF01250D8B49FEF9CF0A1EF9CF0B1EF37
:103940009CF01A1E191E181E171E161E151E141E78
:10395000136C000E14221522162217221822192287
:103960001A2213C001F014C002F015C003F016C0F3
:1039700004F017C005F018C006F019C007F01AC00F
:1039800008F01200000E116E000E106E000E0F6E89
:10399000000E0E6ECEEF9CF0084A092A600023F05C
:1039A000F6FF600027F0F7FF000EF86E0800F550F4
:1039B000200AD8B4DEEF9CF0E0EF9CF0CCEF9CF056
:1039C000F70E0A6EFF0E0B6E600023F0F6FF60002C
:1039D00027F0F7FF000EF86E0800F5500C6E0D6A28
:1039E0000A500C260B500D220D5009E1050E0C5CFF
:1039F000D8A0FDEF9CF0FFEF9CF0CCEF9CF009EF1E
:103A00009DF0000E0F6E010E0E6E084A092A46EF59
:103A10009DF0600023F0F6FF600027F0F7FF000E36
:103A2000F86E0800F5500A6E0B6A0B50000AD8B405
:103A30001CEF9DF046EF9DF00A502B0AD8B405EF1D
:103A40009DF0060AD8B401EF9DF046EF9DF010C03E
:103A500001F011C002F0000E046E0A0E036E61EC5C
:103A6000B0F0600023F0F6FF600027F0F7FF000ED3
:103A7000F86E0800F550015E000E025A300E012467
:103A8000106E000E0220116E05EF9DF0D00E0A6E32
:103A9000FF0E0B6E600023F0F6FF600027F0F7FFCB
:103AA000000EF86E0800F5500C6E0D6A0A500C26D8
:103AB0000B500D220D5009E10A0E0C5CD8A063EFEB
:103AC0009DF065EF9DF027EF9DF00E500F10D8A4EC
:103AD0006CEF9DF06EEF9DF07CEF9DF010C00AF052
:103AE00011C00BF00A1E0B1E0A4A0B2A0AC008F06E
:103AF0000BC009F080EF9DF010C008F011C009F074
:103B00001200000E126E08BE8AEF9DF088EF9DF045
:103B10009CEF9DF0081E071E061E051E041E031EB8
:103B2000021E016C000E022203220422052206223C
:103B300007220822010E126E10BEA3EF9DF0A1EF26
:103B40009DF0B3EF9DF0101E0F1E0E1E0D1E0C1EDD
:103B50000B1E0A1E096C000E0A220B220C220D22DB
:103B60000E220F22102209500A100B100C100D10FB
:103B70000E100F101010D8B4C0EF9DF0C2EF9DF0E2
:103B80000AEF9EF0010E116ED0EF9DF0D89009362D
:103B90000A360B360C360D360E360F361036112A15
:103BA00010AED5EF9DF0D7EF9DF0C6EF9DF0095018
:103BB000015C0A5002580B5003580C5004580D5029
:103BC00005580E5006580F50075810500858D8A0E6
:103BD000ECEF9DF0EEEF9DF0FEEF9DF00950015EE1
:103BE0000A50025A0B50035A0C50045A0D50055AF1
:103BF0000E50065A0F50075A1050085AD8901032DB
:103C00000F320E320D320C320B320A320932112EC3
:103C1000D7EF9DF01250D8B410EF9EF012EF9EF047
:103C200022EF9EF0081E071E061E051E041E031E20
:103C3000021E016C000E022203220422052206222B
:103C40000722082201C001F002C002F003C003F005
:103C500004C004F005C005F006C006F007C007F078
:103C600008C008F012002E0ED5ECB0F0110E226E36
:103C70003C0E216ECB0EE82EFED7212EFCD7222E35
:103C8000FAD700F0310ED5ECB0F0000E1D6E300EFC
:103C9000B7ECA7F0680E216EE40EE82EFED7212EB9
:103CA000FCD700D0320ED5ECB0F0000E1D6E300EF9
:103CB000B7ECA7F0150E216EC60EE82EFED7212E0A
:103CC000FCD700D0330ED5ECB0F0000E1D6E300ED8
:103CD000B7ECA7F0150E216EC60EE82EFED7212EEA
:103CE000FCD700D0340ED5ECB0F0000E1D6E250EC2
:103CF000B7ECA7F0150E216EC60EE82EFED7212ECA
:103D0000FCD700D0350ED5ECB0F0010E1D6E280E9C
:103D1000B7ECA7F0150E216EC60EE82EFED7212EA9
:103D2000FCD700D0360ED5ECB0F0010E1D6E080E9B
:103D3000B7ECA7F0150E216EC60EE82EFED7212E89
:103D4000FCD700D0370ED5ECB0F0010E1D6E010E81
:103D5000B7ECA7F0030E226E080E216E770EE82E48
:103D6000FED7212EFCD7222EFAD700F0380ED5EC44
:103D7000B0F0010E1D6E060EB7ECA7F0150E216E09
:103D8000C60EE82EFED7212EFCD700D0390ED5EC7A
:103D9000B0F0010E1D6E0C0EB7ECA7F0150E216EE3
:103DA000C60EE82EFED7212EFCD700D0410ED5EC52
:103DB000B0F0120051ECB1F00009D8B4E2EF9EF07F
:103DC000E4EF9EF020EF9FF0F1EF9EF09FECB1F05A
:103DD0006CEF9FF0F5ECB1F06CEF9FF0000E6CEF24
:103DE0009FF018C10CF019C10DF020EE09F102D8B6
:103DF00004EF9FF00500FA6EDE50FD6EDE50FE6EA1
:103E0000DE50FF6EFA5012000E6E0F6A0F50000A5D
:103E1000D8B40DEF9FF0EEEF9EF00E50010AD8B42B
:103E2000EEEF9EF0030AD8B4E6EF9EF0010AD8B494
:103E3000EAEF9EF0070AD8B4EEEF9EF0EEEF9EF0A8
:103E400046ECB1F00009D8B428EF9FF02AEF9FF0BC
:103E50006BEF9FF001012951030B0009D8B433EF38
:103E60009FF035EF9FF041EF9FF0010E0E6E29514C
:103E7000030B0F6E0E500F5E29510F18FC0B0F181D
:103E8000296F60008FF4D9FF600093F4DAFFDF50F0
:103E9000126E234B242B2507D8A026072551261167
:103EA000D8A455EF9FF057EF9FF05FEF9FF080ECA5
:103EB000A8F00E6E0E50106E116A63EF9FF0000EA8
:103EC000116E030E106E10C013F01250B2ECB1F070
:103ED00013506CEF9FF0030E1200033404340A6E8B
:103EE0000A50D8A476EF9FF078EF9FF082EF9FF012
:103EF000000E016E000E026E000E036E000E046EC8
:103F0000EFEF9FF001C005F002C006F003C007F01C
:103F100004C008F0200E92EF9FF0D89008320732CC
:103F200006320532E82E8DEF9FF00550096E038EA4
:103F3000FF0E0116FF0E0216FF0E0316000E0416EA
:103F4000960E0A5E0ABEA9EF9FF0A7EF9FF0BFEFA3
:103F50009FF00A50800A970FD8B0B1EF9FF0B3EFEF
:103F60009FF0B5EF9FF078EF9FF0D89004320332C6
:103F7000023201320A3EB5EF9FF0D7EF9FF01F0EDD
:103F80000A64C5EF9FF0C7EF9FF0CFEF9FF078EF87
:103F90009FF0D89001360236033604360A060A50DE
:103FA000D8A4D5EF9FF0D7EF9FF0C9EF9FF009504D
:103FB000D8B4DDEF9FF0DFEF9FF0E7EF9FF0041E36
:103FC000031E021E016C000E02220322042201C005
:103FD00001F002C002F003C003F004C004F01200BC
:103FE000000E2814306E000E2914316E800E2A1433
:103FF000326E7F0E2B14336E30503110321033106E
:10400000D8A405EFA0F007EFA0F00FEFA0F0000E8E
:10401000286E000E296E000E2A6E000E2B6E000E0A
:104020002C14306E000E2D14316E800E2E14326E54
:104030007F0E2F14336E3050311032103310D8A44D
:1040400024EFA0F026EFA0F02EEFA0F0000E2C6ED3
:10405000000E2D6E000E2E6E000E2F6E2BAE33EF67
:10406000A0F035EFA0F03EEFA0F0286C291ED8B0EC
:10407000292A2A1ED8B02A2A800E2B562FAE43EFAB
:10408000A0F045EFA0F04EEFA0F02C6C2D1ED8B0A4
:104090002D2A2E1ED8B02E2A800E2F56000E281A3A
:1040A000000E291A000E2A1A800E2B1A000E2C1A46
:1040B000000E2D1A000E2E1A800E2F1A2C50285C7E
:1040C0002D5029582E502A582F502B58D8B06BEF0E
:1040D000A0F06DEFA0F070EFA0F0D89071EFA0F01D
:1040E000D88012004EC10BF04FC10CF050C10DF042
:1040F00051C10EF001C00BF002C00CF003C00DF076
:1041000004C00EF00BC005F00CC006F00DC007F0A7
:104110000EC008F0180E92EFA0F0D89008320732C7
:1041200006320532E82E8DEFA0F00550096E0A6ABE
:1041300009500A10D8A49FEFA0F0A1EFA0F0C1EFA2
:10414000A0F0D8900B34056E0C34066E0D34076E5B
:104150000E34086E0550061007100810D8A4B3EFEF
:10416000A0F0B5EFA0F0BBEFA0F0000E026E020EC3
:10417000016EF0EFA0F0000E026E030E016EF0EF84
:10418000A0F009280A10D8A4C8EFA0F0CAEFA0F048
:10419000ECEFA0F00BC005F00CC006F00DC007F06E
:1041A0000EC008F0090ED8900536063607360836D8
:1041B000E82ED3EFA0F00550061007100810D8B471
:1041C000E4EFA0F0E7EFA0F0010EE8EFA0F0000EA2
:1041D000016E026AF0EFA0F0000E026E040E016E96
:1041E000120001C008F002C009F003C00AF004C0C8
:1041F0000BF00506D8A00606052806E10628D8A477
:1042000004EFA1F006EFA1F013EFA1F0000E026E93
:10421000000E016E6DEFA1F0084A092A0A4A0B2A26
:104220000506D8A00606600023F0D9FF600027F03D
:10423000DAFFDF50D8B41FEFA1F021EFA1F056EF65
:10424000A1F060002BF0F6FF60002FF0F7FF000EEA
:10425000F86E0800F5500009D8B431EFA1F033EF43
:10426000A1F056EFA1F005500610D8B43AEFA1F036
:104270003CEFA1F056EFA1F0600023F0D9FF600001
:1042800027F0DAFFDF50076E60002BF0F6FF6000CA
:104290002FF0F7FF000EF86E0800F5500718D8B49D
:1042A00054EFA1F056EFA1F00CEFA1F0600023F065
:1042B000D9FF600027F0DAFFDF50076E60002BF0B7
:1042C000F6FF60002FF0F7FF000EF86E0800F550C3
:1042D000075C016E026AD8A00206120049ECAEF03B
:1042E000330E62ECAFF0000E0001B96FBC0EB925C1
:1042F000D96EDA6A010EDA22A2ECAEF0DF6E0001AE
:10430000B92B070EB96587EFA1F089EFA1F076EF21
:10431000A1F0280E0101BC19D8A491EFA1F093EFF0
:10432000A1F099EFA1F06F0E076EFE0E086EF3EC90
:10433000ABF0B10E076EFF0E086EF3ECABF0010EA2
:104340000001B96FA00EAC6F020EAD6FE50EAE6F3F
:10435000FF0EAF6FBC0EB925D96EDA6A010EDA22F4
:10436000DF505F6E5F50B06FB16BC3ECACF0A00E6E
:10437000016E020E026E28ECAAF00001B92B070EA6
:10438000B965C5EFA1F0C7EFA1F0A2EFA1F0F1EC84
:10439000AFF0BC0E016E010E026E070E036E60ECF4
:1043A000AAF00001B86FA00EAC6F020EAD6F860EC2
:1043B000AE6FFF0EAF6FB8C0B0F0B16BC3ECACF036
:1043C000A00E016E020E026E28ECAAF0F1ECAFF026
:1043D000120020EE11F0070EDE6AE806FDE2095039
:1043E0000A100B100C100D100E100F101010D8B476
:1043F000FCEFA1F0FEEFA1F050EFA2F0010E196E5C
:104400000CEFA2F0D89009360A360B360C360D3672
:104410000E360F361036192A10AE11EFA2F013EF38
:10442000A2F002EFA2F0D8901136123613361436ED
:1044300015361636173618360950015C0A500258E0
:104440000B5003580C5004580D5005580E50065888
:104450000F50075810500858D8A031EFA2F033EF92
:10446000A2F044EFA2F00950015E0A50025A0B502C
:10447000035A0C50045A0D50055A0E50065A0F504C
:10448000075A1050085A1180D89010320F320E324D
:104490000D320C320B320A320932192E13EFA2F010
:1044A00011C001F012C002F013C003F014C004F0F8
:1044B00015C005F016C006F017C007F018C008F0C8
:1044C000120020EE2EF0080EDE6AE806FDE249EC4E
:1044D000AEF0550E62ECAFF0000E3B6E3B50282460
:1044E000D96E000E2920DA6EDF5062ECAFF03B2A65
:1044F000070E3B647EEFA2F080EFA2F06EEFA2F019
:10450000BE0E62ECAFF0000E3B6E2E0E3B24D96E59
:10451000DA6A000EDA22A2ECAEF0DF6E3B2A010E60
:104520003B6495EFA2F097EFA2F085EFA2F049EC83
:10453000AEF02E502FC02CF02D6A2CC02DF02C6A1E
:104540002C26000E2D222CC001F02DC002F0000EF2
:1045500002BEFF0E036E046E010E24EC9BF001C040
:104560000FF002C010F003C011F004C012F0000EF2
:10457000136E000E146E800E156E3D0E166EB6ECA8
:104580008DF00FC037F010C038F011C039F012C0F4
:104590003AF037C028F038C029F039C02AF03AC0C4
:1045A0002BF012000001C651C711D8A4DAEFA2F017
:1045B000DCEFA2F0E2EFA2F0C6C010F0C7C011F02D
:1045C000E8EFA2F0FF0EC625106EFF0EC721116E98
:1045D000CAA1EDEFA2F0EFEFA2F0F8EFA2F00CC04D
:1045E00001F0026A0AC003F00BC004F03EECA3F035
:1045F00011BEFDEFA2F0FFEFA2F001EFA3F005EF77
:10460000A3F0000E116E000E106E000E0F6E000E65
:104610000E6E17EFA3F0000E026E200E016E0AC0A0
:1046200003F00BC004F03EECA3F00E4A0F2A10502A
:104630000E5C0F50800A0D6E1150800A0D58D8A0E4
:1046400024EFA3F026EFA3F00BEFA3F00001CAB113
:104650002CEFA3F02EEFA3F037EFA3F00CC001F086
:10466000026A0AC003F00BC004F03EECA3F0010E96
:104670000E240A6E000E0F200B6E12000350041061
:10468000D8B445EFA3F047EFA3F050EFA3F00350E9
:104690000410D8A44EEFA3F050EFA3F055EFA3F011
:1046A0000150FCECB1F0A9EFA3F020EE09F00350AB
:1046B000D9260450DA22DE50DE10D8B462EFA3F01F
:1046C00064EFA3F07FEFA3F020EE09F00350D926AA
:1046D0000450DA2210EE03F00350E1260450E222E7
:1046E000DE50E65CE650800A096EDE50800A09580A
:1046F000D8B07DEFA3F07FEFA3F0A9EFA3F020EEF9
:1047000003F00350D9260450DA226F0078FF05F039
:104710006F0074FF06F060000FF0D9FF600013F027
:10472000DAFF6F0078FF07F06F0074FF08F00550A4
:104730000724D96E06500820DA6E600007F0DFFF0C
:1047400020EE03F00350D9260450DA22DE2A000EB0
:10475000DD22120009500A100B100C100D100E1063
:104760000F101010D8B4B7EFA3F0B9EFA3F001EF1A
:10477000A4F0010E116EC7EFA3F0D89009360A36E7
:104780000B360C360D360E360F361036112A10AE9B
:10479000CCEFA3F0CEEFA3F0BDEFA3F00950015C86
:1047A0000A5002580B5003580C5004580D5005582D
:1047B0000E5006580F50075810500858D8A0E3EF75
:1047C000A3F0E5EFA3F0F5EFA3F00950015E0A5066
:1047D000025A0B50035A0C50045A0D50055A0E50F1
:1047E000065A0F50075A1050085AD89010320F32FC
:1047F0000E320D320C320B320A320932112ECEEF4C
:10480000A3F001C001F002C002F003C003F004C035
:1048100004F005C005F006C006F007C007F008C0A8
:1048200008F012000001CAA118EFA4F01AEFA4F0DA
:1048300024EFA4F013C00AF014C00BF011C00CF068
:1048400012C00DF0E8ECADF016BE29EFA4F02BEF8E
:10485000A4F031EFA4F015C01AF016C01BF035EF2C
:10486000A4F0000E1B6E000E1A6E000E196E000EE4
:10487000186E47EFA4F0000E026E200E016E11C0FC
:1048800003F012C004F03EECA3F0184A192A1A50A3
:10489000185C1950800A176E1B50800A1758D8A050
:1048A00054EFA4F056EFA4F03BEFA4F00001CAB11E
:1048B0005CEFA4F05EEFA4F068EFA4F013C00AF080
:1048C00014C00BF011C00CF012C00DF0E8ECADF00C
:1048D00013C001F014C002F085ECAEF01A500124B0
:1048E000116E1B500220126E1200000E066E04BEE6
:1048F0007EEFA4F07CEFA4F084EFA4F0036C041E20
:10490000D8B0042A010E066E02BE8BEFA4F089EF28
:10491000A4F091EFA4F0016C021ED8B0022A010E9F
:10492000061A000E086E000E076E03500410D8B46D
:104930009CEFA4F09EEFA4F0C6EFA4F0010E056E6C
:10494000A6EFA4F0D89003360436052A04AEABEFE8
:10495000A4F0ADEFA4F0A2EFA4F0D890073608368B
:104960000350015C04500258D8A0B9EFA4F0BBEF8B
:10497000A4F0C0EFA4F00350015E0450025A078077
:10498000D89004320332052EADEFA4F00650D8B40F
:10499000CCEFA4F0CEEFA4F0D2EFA4F0076C081E89
:1049A000D8B0082A07C001F008C002F0120011EFC9
:1049B000A5F0800EFDECA8F0540E1F6EFD0E206ECB
:1049C0003BECA9F0800EFDECA8F02FEFA5F0C00E97
:1049D000FDECA8F0540E1F6EFD0E206E3BECA9F00E
:1049E000C00EFDECA8F02FEFA5F0940EFDECA8F0A2
:1049F000D50E1F6EFE0E206E3BECA9F0940EFDEC62
:104A0000A8F02FEFA5F0D40EFDECA8F0D50E1F6E88
:104A1000FE0E206E3BECA9F0D40EFDECA8F02FEFBB
:104A2000A5F024C026F025C027F02750000AD8B4EE
:104A30001CEFA5F02FEFA5F02650010AD8B4D9EF4E
:104A4000A4F0030AD8B4E7EFA4F0010AD8B4F5EF54
:104A5000A4F0070AD8B403EFA5F02FEFA5F0D00E0D
:104A6000266ECA0EE82EFED7262EFCD71200000EA8
:104A7000066E02BE40EFA5F03EEFA5F046EFA5F0B2
:104A8000016C021ED8B0022A010E066E04BE4DEF64
:104A9000A5F04BEFA5F051EFA5F0036C041ED8B0C4
:104AA000042A03500410D8B458EFA5F05AEFA5F02B
:104AB0007EEFA5F0010E056E62EFA5F0D8900336EB
:104AC0000436052A04AE67EFA5F069EFA5F05EEFA6
:104AD000A5F00350015C04500258D8A072EFA5F075
:104AE00074EFA5F078EFA5F00350015E0450025A70
:104AF000D89004320332052E69EFA5F00650D8B4E1
:104B000084EFA5F086EFA5F08AEFA5F0016C021EF8
:104B1000D8B0022A01C001F002C002F01200000E5B
:104B20000114096E000E02140A6E800E03140B6E3F
:104B30007F0E04140C6E09500A100B100C10D8A430
:104B4000A4EFA5F0A6EFA5F0AEEFA5F0000E016E64
:104B5000000E026E000E036E000E046E000E0514B1
:104B6000096E000E06140A6E800E07140B6E7F0E7F
:104B700008140C6E09500A100B100C10D8A4C3EFC7
:104B8000A5F0C5EFA5F0CDEFA5F0000E056E000E67
:104B9000066E000E076E000E086E055001180FE13C
:104BA000065002180CE10750031809E108500418D8
:104BB000D8B4DDEFA5F0DFEFA5F0E2EFA5F0D890D7
:104BC000E3EFA5F0D8801200016E010E026E010124
:104BD00029B7EDEFA5F0EFEFA5F034EFA6F001C097
:104BE00022F129952987FC0E29170F0E276F010E38
:104BF000216FF40E206F2989F20E006F630E016F92
:104C0000010E026F000E126F000E136FF20E036F93
:104C1000630E046F010E056F000E146F000E156F0A
:104C2000F20E066F630E076F010E086F000E166F0F
:104C3000000E176FF20E096F630E0A6F010E0B6FF5
:104C4000000E186F000E196FEE0E0C6F630E0D6FD5
:104C5000010E0E6F000E1A6F000E1B6FD1ECB1F03B
:104C600008ECB0F0000E026E02501200010129891A
:104C70005AEFA6F0E4ECB1F0080E87EFA6F0E4ECF2
:104C8000B1F0070E87EFA6F001012529B7ECB1F0CE
:104C9000040E87EFA6F0070E01012719D8B453EFD1
:104CA000A6F055EFA6F057EFA6F0E7ECB1F00F0E27
:104CB00087EFA6F012C10CF013C10DF002D86BEF14
:104CC000A6F00500FA6E0051FD6E0151FE6E025114
:104CD000FF6EFA5012000E6E0F6A0F50000AD8B421
:104CE00074EFA6F04BEFA6F00E50010AD8B44BEFCC
:104CF000A6F0030AD8B43FEFA6F0010AD8B43AEF01
:104D0000A6F0070AD8B444EFA6F04BEFA6F01200C5
:104D10005CECB1F00009D8A490EFA6F092EFA6F0F9
:104D200095EFA6F0040ED6EFA6F001012951030B72
:104D30000009D8B49EEFA6F0A0EFA6F0ACEFA6F065
:104D4000010E106E2951030B116E1050115E295186
:104D50001118FC0B1118296F2507D8A0260725511B
:104D60002611D8B4B6EFA6F0B8EFA6F0C6EFA6F0BD
:104D7000E1ECB1F060008FF4D9FF600093F4DAFF4A
:104D8000DF6E0101234B242B92EFA6F036ECA6F048
:104D9000126EE1ECB1F060008FF4D9FF600093F483
:0E4DA000DAFFDF6E0101234B242B12501200AC
:104DB0003901A3A7DEEFA6F0E0EFA6F024EFA7F0FD
:104DC00093A7E5EFA6F0E7EFA6F024EFA7F06F00BA
:104DD000A0F7FDF00D0E0001FD19D8B4F2EFA6F01A
:104DE000F4EFA6F0FFEFA6F0E15109E1800EE05DDF
:104DF000D8A0FDEFA6F0FFEFA6F015EFA7F0010E8B
:104E0000F86F000EE025D96E020EE121DA6E000E79
:104E1000DF6EE0C0E2F0E1C0E3F0000EE16F000EF3
:104E2000E06F3901939724EFA7F0000EE025D96ECB
:104E3000020EE121DA6E6000F7F3DFFFE04BE12BB9
:104E4000E0C0E2F0E1C0E3F0110022500001FE5D9D
:104E5000FF51800A256E2350800A2558D8B033EFC1
:104E6000A7F035EFA7F039EFA7F0FEC022F0FFC0A2
:104E700023F020042110D8A440EFA7F042EFA7F0C0
:104E800046EFA7F022507F0FFDECA8F0020E20188D
:104E90002110D8A44EEFA7F050EFA7F054EFA7F0E1
:104EA0002250BF0FFDECA8F0030E266E080E256EF3
:104EB000770EE82EFED7252EFCD7262EFAD700F047
:104EC0002450BFECA8F0030E266E080E256E770E58
:104ED000E82EFED7252EFCD7262EFAD700F012009A
:104EE000066E015002100310D8B479EFA7F07BEFE3
:104EF000A7F09CEFA7F00650030D000EF324D96E27
:104F0000010EF420DA6E600007F0DEFF60000BF0A7
:104F1000DEFF60000FF0DEFF0650020D120EF324DC
:104F2000D96E010EF420DA6E600013F0DEFF60002F
:104F300017F0DDFFB6EFA7F00650030D000EF324C7
:104F4000D96E010EF420DA6EF20EDE6E630EDE6EA6
:104F5000010EDE6E0650020D120EF324D96E010E04
:104F6000F420DA6E000EDE6E000EDD6E12001F6E93
:104F70001F50F00B0C09206E20C01BF00001F651F1
:104F800076ECB0F0500EE82EFED71F50F00B08095B
:104F9000206E20C01BF00001F65176ECB0F0500EF0
:104FA000E82EFED71D04D8A4D8EFA7F0DAEFA7F0BB
:104FB000FCEFA7F01FC01EF00F0E1E161E38F00BE0
:104FC0000C09206E20C01BF00001F65176ECB0F009
:104FD000500EE82EFED71FC01EF00F0E1E161E38F4
:104FE000F00B0809206E20C01BF00001F65176EC92
:104FF000B0F0500EE82EFED71200000EBA6E000E72
:10500000BB6E000EBC6EC268D70EC36E870EC46E38
:10501000000E3A01606F000E506F000E406F000EE0
:10502000816F3F0E516FFE0E416FC00E616F000E1B
:105030005A6F000E5B6F000E6A6F000E6B6F010EF1
:10504000426F000E526F180E626F436953696369B5
:10505000446954696469080E846F000E476F000E3E
:10506000466F000E456F140EE26F210E136F220E75
:10507000146F130E166F170EE56F130EE16F12000B
:10508000CA0EF66E610EF76E010EF86E00EEC8F1F4
:1050900010EE1EF009006F00D7FFEEFFE550E15063
:1050A000F9E1F60EF66E630EF76E010EF86E09006A
:1050B0006F00D4FFFEF009006F00D4FFFFF000EE98
:1050C00000F3800EEE6AE806FDE100EE00F2F00E5D
:1050D000EE6AE806FDE100EE00F1C80EEE6AE806B1
:1050E000FDE100EEC0F03E0EEE6AE806FDE1080EBE
:1050F000D56E000ED66E000ED76E0001AAEF91F0AD
:105100000101298995EFA8F0E4ECB1F0070EBEEF9C
:10511000A8F001012529B7ECB1F0030EBEEFA8F00D
:10512000E7ECB1F00A0EBEEFA8F012C10CF013C10B
:105130000DF002D8A6EFA8F00500FA6E0051FD6E42
:105140000151FE6E0251FF6EFA5012000E6E0F6A90
:105150000F50000AD8B4AFEFA8F090EFA8F00E50AF
:10516000010AD8B490EFA8F0030AD8B484EFA8F0ED
:10517000060AD8B489EFA8F090EFA8F012001E6ECE
:105180001E50F00B0D090001F26FF2C01BF0F6513A
:1051900076ECB0F0500EE82EFED71E50F00B090949
:1051A0000001F26FF2C01BF0F65176ECB0F0500E39
:1051B000E82EFED71EC01DF00F0E1D161D38F00B79
:1051C0000D090001F26FF2C01BF0F65176ECB0F061
:1051D000500EE82EFED71EC01DF00F0E1D161D38F6
:1051E000F00B09090001F26FF2C01BF0F65176ECEA
:1051F000B0F0500EE82EFED712001E6E1E50F00BBF
:105200000C091F6E1FC01BF00001F65176ECB0F0C8
:10521000500EE82EFED71E50F00B08091F6E1FC05F
:105220001BF00001F65176ECB0F0500EE82EFED7E0
:105230001EC01DF00F0E1D161D38F00B0C091F6E41
:105240001FC01BF00001F65176ECB0F0500EE82EB6
:10525000FED71EC01DF00F0E1D161D38F00B0809DD
:105260001F6E1FC01BF00001F65176ECB0F0500E1F
:10527000E82EFED71200000E236E000E226E59EFAC
:10528000A9F060007FF0F6FF600083F0F7FF000EEA
:10529000F86E0800F550BFECA8F01F4A202A224AF9
:1052A000232A150E216EC60EE82EFED7212EFCD71E
:1052B00000D060007FF0F6FF600083F0F7FF000E83
:1052C000F86E0800F5500009D8B469EFA9F06BEF4B
:1052D000A9F077EFA9F00001FE51225CFF5123589D
:1052E000D8A075EFA9F077EFA9F041EFA9F012006F
:1052F000246E2050216E226A21500001FE5DFF5174
:10530000800A236E2250800A2358D8B08AEFA9F071
:105310008CEFA9F08EEFA9F0FE05206E2404D8A42E
:1053200094EFA9F096EFA9F09AEFA9F020507F0F23
:10533000FDECA8F0020E2418D8A4A1EFA9F0A3EF69
:10534000A9F0A7EFA9F02050BF0FFDECA8F0020EC6
:10535000226EA00E216E920EE82EFED7212EFCD7D3
:10536000222EFAD700D01200D1ECB1F0020E0101CA
:10537000286FC7EFA9F09FECB1F0EEEFA9F0F5ECC4
:10538000B1F0EEEFA9F090ECB1F0EEEFA9F014C19E
:105390000CF015C10DF020EE03F102D8DAEFA9F000
:1053A0000500FA6EDE50FD6EDE50FE6EDE50FF6EC2
:1053B000FA5012000E6E0F6A0F50000AD8B4E3EFD5
:1053C000A9F0C3EFA9F00E50020AD8B4BBEFA9F0C0
:1053D000010AD8B4BFEFA9F0C3EFA9F012009AEC0C
:1053E000ACF001012951030B0009D8B4FAEFA9F080
:1053F000FCEFA9F009EFAAF051ECB1F00009D8B424
:1054000004EFAAF006EFAAF009EFAAF0100E0101CE
:10541000276F01012751030D670EF324F66EFB0E73
:10542000F420F76EF86A000EF82202D825EFAAF0F1
:105430000500FA6E0900F550FD6E0900F550FE6E8C
:105440000900F550FF6EFA5012000101276F12009B
:10545000000E0001CF6F000ECE6F51EFAAF03901A0
:10546000A3A935EFAAF037EFAAF02FEFAAF00001B9
:10547000CE510124D96ECF510220DA6EDF503D01AA
:10548000EA6F0001CE4BCF2BCF5109E1810ECE5DEB
:10549000D8A04DEFAAF04FEFAAF051EFAAF05FEFBE
:1054A000AAF0CE510124D96ECF510220DA6EDF501E
:1054B000D8A45DEFAAF05FEFAAF02FEFAAF01200D8
:1054C000000E086E000E066E8CEFAAF00650012446
:1054D000D96E000E0220DA6EDF50056E000E076EE8
:1054E00008500518010B046ED89008320450D8B447
:1054F0007CEFAAF07EEFAAF080EFAAF08C0E081ADB
:10550000D8900532072A070E076489EFAAF08BEFBF
:10551000AAF070EFAAF0062A0350065CD8A093EF19
:10552000AAF095EFAAF066EFAAF008501200FC0E60
:1055300001012917020E286F2995A6EFAAF0F3ECB6
:10554000B1F0CDEFAAF00F0ECDEFAAF016C10CF01E
:1055500017C10DF020EE06F102D8B9EFAAF0050050
:10556000FA6EDE50FD6EDE50FE6EDE50FF6EFA50BB
:1055700012000E6E0F6A0F50000AD8B4C2EFAAF0E4
:10558000A3EFAAF00E50020AD8B49FEFAAF0010AC6
:10559000D8B49FEFAAF0A3EFAAF012004CC050F0CD
:1055A0004DC051F0000E0001C56F000EC46FECEF4E
:1055B000AAF04AC040F04BC041F0500E426E000EBF
:1055C000436E4EC044F04FC045F009EC86F04050A9
:1055D0000001C4274150C523600043F1F6FF60007D
:1055E00047F1F7FF000EF86E0800F5500009D8A447
:1055F000FCEFAAF0FEEFAAF0D9EFAAF0C4C04AF07F
:10560000C5C04BF0120007C00BF008C00CF005C07D
:105610000DF006C00EF00B50096E0C500A6E0B4ACE
:105620000C2A600027F0F6FF60002BF0F7FF000E59
:10563000F86E600037F0D9FF60003BF0DAFF0D4AEA
:105640000E2A1F0EF76403D00800F55007D06F0034
:10565000DBFFE9FF6F00DFFFEAFFEF50DF6EDF5097
:10566000D8A435EFABF037EFABF00BEFABF0120097
:10567000000E236E000E226E49EFABF022501F2465
:10568000D96E23502020DA6EDF50BFECA8F0224AFA
:10569000232A22501F24D96E23502020DA6EDF5097
:1056A000D8B455EFABF057EFABF067EFABF00001BC
:1056B000FE51225C2350800A216EFF51800A21583E
:1056C000D8A065EFABF067EFABF03EEFABF01200A8
:1056D0001A6E1A50E4ECA5F00009D8B472EFABF0E2
:1056E00074EFABF069EFABF016C001F017C002F039
:1056F00018C003F019C004F0B2ECB0F0000E076E51
:10570000000E086E000E096E000E0A6E000E0B6E83
:1057100012ECB1F0C1ECB1F036ECB0F0E806D8B460
:1057200094EFABF096EFABF08CEFABF012003901D9
:10573000A3A19DEFABF09FEFABF0A1EFABF0C4EFF7
:10574000ABF0A2AFA6EFABF0A8EFABF0AAEFABF0D7
:10575000C4EFABF03D0179A5B0EFABF0B2EFABF029
:10576000B4EFABF0C4EFABF079AFB9EFABF0BBEF98
:10577000ABF0BDEFABF0C4EFABF076A9C2EFABF08E
:0A578000C4EFABF097EFABF012009E
:10578C003901A9A1CCEFABF0CEEFABF0F2EFABF05F
:10579C0099A1D3EFABF0D5EFABF0F2EFABF000018A
:1057AC00D3BFE1EFABF0D35108E1D205D8A0E1EFC4
:1057BC00ABF0E3EFABF0E8EFABF0D207D8A0D30738
:1057CC00EBEFABF0F58B39019991000E0101616F94
:1057DC00010E606F3901A99111000BEFACF039018A
:1057EC00A3A9FBEFABF0FDEFABF0F5EFABF0600076
:1057FC001FF0F6FF600023F0F7FF000EF86E0800B4
:10580C006F00D7FFEAFD074A082A60001FF0F6FF79
:10581C00600023F0F7FF000EF86E0800F550000949
:10582C00D8A41BEFACF01DEFACF0F5EFABF0120011
:10583C00046E000E0001D16F000ED06F35EFACF08E
:10584C00520E026E2B0E016E000EE82EFED7012EAC
:10585C00FCD7022EFAD700D00001D04BD12B04502C
:10586C00016E026A0150D05DD151800A036E025064
:10587C00800A0358D8A045EFACF047EFACF026EF08
:10588C00ACF01200010E076E200E01180210D8B4F5
:10589C0052EFACF054EFACF06DEFACF0F70E036ED2
:1058AC00FF0E046E01C005F002C006F00350052681
:1058BC0004500622065009E1050E055CD8A069EFDC
:1058CC00ACF06BEFACF06DEFACF0000E076E07C0F8
:1058DC0001F0026A1200146E010E156E010129B559
:1058EC007AEFACF07CEFACF098EFACF02985000EC1
:1058FC00156E2551B7ECB1F01450D8B488EFACF05C
:10590C008AEFACF091EFACF0040E0101276F1FECA5
:10591C00B0F096EFACF0030E0101276F3BECB1F049
:10592C00F4ECB0F0155012007DECB1F00009D8B4D5
:10593C00A2EFACF0A4EFACF0A8EFACF0F0ECB1F04F
:10594C00C2EFACF067ECB1F00009D8B4B0EFACF03A
:10595C00B2EFACF0B6EFACF0EAECB1F0C2EFACF0F9
:10596C0072ECB1F00009D8B4BEEFACF0C0EFACF003
:10597C00C2EFACF0EDECB1F01200B00E526E000EB6
:10598C00536EACC054F0ADC055F0000E586E000E06
:10599C00576E000E5E6E000E5D6E540E4A6E000E5B
:1059AC004B6EAEC04CF0AFC04DF0520E4E6E000EB2
:1059BC004F6ECEECAAF057500001AC25D96E585062
:1059CC00AD21DA6E000EDF6E120020EE02F00C50EC
:1059DC00D9260D50DA226F0078FF01F06F0074FFAA
:1059EC0002F0600033F0D9FF600037F0DAFF6F008F
:1059FC0078FF03F06F0074FF04F0B2ECB0F0000E0F
:105A0C00076E000E086E000E096E000E0A6E000E78
:105A1C000B6E20ECB1F0020E1200010E0114016E9F
:105A2C00026A01500210D8B41EEFADF020EFADF0B9
:105A3C002DEFADF0C290CA901A0EE82EFED700D012
:105A4C00C280C00E00D0E82EFDD738EFADF0C2906A
:105A5C00CA90E00E00D0E82EFDD7C2800A0EE82EC8
:105A6C00FED700D01200000E3D01EC6F000EED6F62
:105A7C00000EEE6F000EEF6F000EF06F000EF16F68
:105A8C00B00EF26F800EF36F000EF46F8A0EF56F8E
:105A9C00000EF66F000EF76F000EF86F000EF96F28
:105AAC00000EFA6FF28BF289390193971200BF0E38
:105ABC00096EFF0E0A6E07C00BF008C00CF00950FF
:105ACC000B260A500C220C5007E11A0E0B5CD8B0B6
:105ADC0072EFADF074EFADF07BEFADF0200E071070
:105AEC00076E0850086E7FEFADF007C007F008C0D6
:105AFC0008F01200000E2C1A000E2D1A000E2E1A91
:105B0C00800E2F1A28C001F029C002F02AC003F021
:105B1C002BC004F02CC005F02DC006F02EC007F0F1
:105B2C002FC008F056EC8BF001C028F002C029F011
:105B3C0003C02AF004C02BF01200026E800E036E1C
:105B4C00BDEFADF0025003140009D8B4B0EFADF0C6
:105B5C00B2EFADF0B7EFADF02A0ED5ECB0F0BAEF76
:105B6C00ADF0200ED5ECB0F0D8900330036E03509E
:105B7C00D8A4C3EFADF0C5EFADF0A8EFADF01200B7
:105B8C009F0E096EFF0E0A6E07C00BF008C00CF0DA
:105B9C0009500B260A500C220C5007E11A0E0B5C14
:105BAC00D8B0DBEFADF0DDEFADF0E3EFADF05F0EB5
:105BBC000714076E086AE7EFADF007C007F008C0DE
:105BCC0008F01200000E106E000E0F6EF9EFADF023
:105BDC000EC001F0026A0CC003F00DC004F03EECE4
:105BEC00A3F00F4A102A0F500A24D96E10500B2024
:105BFC00DA6EDF500E6E0E50D8A407EFAEF009EF40
:105C0C00AEF0EEEFADF0120014BE17EFAEF0145084
:105C1C0006E11304D8B015EFAEF017EFAEF025EF98
:105C2C00AEF013C015F014C016F0151E161E154A52
:105C3C00162A15C013F016C014F029EFAEF013C0DD
:105C4C0013F014C014F01200600007F0D9FF6000CC
:105C5C000BF0DAFF014A022ADF50056E60000FF0EC
:105C6C00F6FF600013F0F7FF034A042A000EF86EEB
:105C7C000800F5500518D8B446EFAEF048EFAEF07A
:105C8C002AEFAEF01200C290CA900A0E016EF80E06
:105C9C00E82EFED7012EFCD700D0C280C00E00D05B
:105CAC00E82EFDD7CAB05DEFAEF05FEFAEF066EF59
:105CBC00AEF0E40E00D000D0E82EFCD700D000D01F
:105CCC0012009F0E036EFF0E046E200E0110056E67
:105CDC00000E0210066E03500526045006220650D4
:105CEC000AE11A0E055CD8A07EEFAEF081EFAEF0A3
:105CFC00010E82EFAEF0000E016E026A120001C0BE
:105D0C0003F002C004F08DEFAEF0014A022A6000ED
:105D1C0007F0D9FF60000BF0DAFFDF50D8A499EF41
:105D2C00AEF09BEFAEF08BEFAEF00350015C016E6A
:105D3C0004500258026E1200000E026E000E036E2A
:105D4C00D89002324CECB0F00009D8B4B0EFAEF001
:105D5C00B2EFAEF0B3EFAEF0028E032A070E03647F
:105D6C00BAEFAEF0BCEFAEF0A6EFAEF00250120000
:105D7C009F0E036EFF0E046E01C005F002C006F00C
:105D8C00035005260450062206500AE11A0E055C43
:105D9C00D8A0D3EFAEF0D6EFAEF0010ED7EFAEF049
:105DAC00000E016E026A1200BF0E036EFF0E046E2F
:105DBC0001C005F002C006F003500526045006226F
:105DCC0006500AE11A0E055CD8A0EFEFAEF0F2EF28
:105DDC00AEF0010EF3EFAEF0000E016E026A12008F
:105DEC000150021003100410D8B4FFEFAEF001EF15
:105DFC00AFF009EFAFF0000E011A000E021A000E00
:105E0C00031A800E041A01C001F002C002F003C094
:105E1C0003F004C004F01200D00E036EFF0E046EEB
:105E2C0001C005F002C006F00350052604500622FE
:105E3C0006500AE10A0E055CD8A027EFAFF02AEF56
:105E4C00AFF0010E2BEFAFF0000E016E026A1200E4
:105E5C000001D451D511D8A436EFAFF038EFAFF024
:105E6C003FEFAFF0B290390194910001F58342EF0E
:105E7C00AFF0D407D8A0D507CF0EB16E2C0EB06EF4
:105E8C003901A49111003D017995600007F06EFD78
:105E9C00000E6C6F738B79A556EFAFF058EFAFF027
:105EAC0051EFAFF074AB5DEFAFF060EFAFF0010E00
:105EBC0061EFAFF0000E1200046E000E056E04C010
:105ECC0003F0010E03160350016E026A13ECADF0E1
:105EDC00D8900432052A070E056477EFAFF079EFFE
:105EEC00AFF065EFAFF012000CC001F00DC002F086
:105EFC00000E046E010E036EB2ECB0F0000E076ED5
:105F0C00000E086E000E096E000E0A6E000E0B6E6F
:105F1C0020ECB1F0040E12000CC001F00DC002F028
:105F2C00000E046E020E036EB2ECB0F0000E076EA3
:105F3C00000E086E000E096E000E0A6E000E0B6E3F
:105F4C0020ECB1F0020E12000CC001F00DC002F0FA
:105F5C00000E046E010E036EB2ECB0F0000E076E74
:105F6C00000E086E000E096E000E0A6E000E0B6E0F
:105F7C0020ECB1F0020E12000CC001F00DC002F0CA
:105F8C00000E046E020E036EB2ECB0F0000E076E43
:105F9C00000E086E000E096E000E0A6E000E0B6EDF
:105FAC0020ECB1F0040E12000FC001F010C002F092
:105FBC0085ECAEF001500F24056E02501020066ED9
:105FCC0011C007F012C008F003ECABF00FC00FF0DB
:105FDC0010C010F012003901A3A9F7EFAFF0F9EFE0
:105FEC00AFF0F1EFAFF00D0E3D01EA6F3901A3A94F
:105FFC0002EFB0F004EFB0F0FCEFAFF00A0E3D0191
:10600C00EA6F12003D0173BF0EEFB0F010EFB0F06D
:10601C001EEFB0F0000E796F000E7A6F000E766FE7
:10602C006C69510E3A016A6F510E6B6F3D01738FA3
:10603C00120001012951FC0B0209296F25052611BB
:10604C00D8A42BEFB0F02DEFB0F02FEFB0F036EC72
:10605C00A6F0D88001012235B2ECB1F0040E12008A
:10606C00010E016E010129B53EEFB0F040EFB0F02A
:10607C004AEFB0F029972269D1ECB1F003ECB1F002
:10608C00ACECB1F028C101F001501200C290CA90E2
:10609C00050EE82EFED700F0C2801A0EE82EFED7B1
:1060AC0000D0000ECAB0010E016EB00E00D0E82E6A
:1060BC00FDD701501200015003026F00CCFF05F018
:1060CC006F00D0FF06F001500402F3500626025078
:1060DC000302F350062605C001F006C002F01200C0
:1060EC001C6E1BC0C4F1000E0101C56FC40E166EF0
:1060FC00010E176E000E196E010E186E1C5068EC16
:10610C00ABF0A00EE82EFED71200D8ECB1F0D5EC17
:10611C00B1F00009D8B495EFB0F097EFB0F09DEF67
:10612C00B0F0000EB7ECB1F0000EB2ECB1F0000E16
:10613C00120049ECAEF0CC0E62ECAFF0440E62EC07
:10614C00AFF04CECB0F00009D8B4AFEFB0F0B1EF59
:10615C00B0F0A7EFB0F01200010129A9B8EFB0F030
:10616C00BAEFB0F0C3EFB0F001C023F102C024F1DC
:10617C0003C025F104C026F129991200030E3D013C
:10618C007B6F040E736F800E746F000E756F000EB4
:10619C006C6F7599200E6E6F7995739F1200016E5E
:1061AC00D9EFB0F000F03901A3A9DFEFB0F0E1EFC7
:1061BC00B0F0D8EFB0F0600007F0EAFD12005EFC22
:1061CC00B0FBEEFC35FD16FD65FDC1FC77FD91FCC9
:1061DC0075FD0102030405060708D4FFFAEFB0F0C1
:1061EC0097ECABF0EFECA9F0010129B500EFB1F0A1
:1061FC0002EFB1F0F6EFB0F01200390193939395E2
:10620C00929F93913D017A917A957A9F7A9D7A9398
:10621C00769376957691120007C001F008C002F0D3
:10622C0009C003F00AC004F00BC005F0020E70ECBC
:10623C00A7F0120007C001F008C002F009C003F07B
:10624C000AC004F00BC005F0000E70ECA7F01200B1
:10625C00286E25C020F0285078ECA9F026C01FF03D
:10626C0027C020F038ECABF0120001012951FC0BD7
:10627C000209296F22512225B2ECB1F0030E120053
:10628C003D0178BB4CEFB1F04FEFB1F0010E50EF88
:10629C00B1F0000E12003D0174BB57EFB1F05AEF94
:1062AC00B1F0010E5BEFB1F0000E12003D0178B1C0
:1062BC0062EFB1F065EFB1F0010E66EFB1F0000ED8
:1062CC0012003D0179B56DEFB1F070EFB1F0010E38
:1062DC0071EFB1F0000E12003D0176B978EFB1F01C
:1062EC007BEFB1F0010E7CEFB1F0000E12003D011E
:1062FC0079BF83EFB1F086EFB1F0010E87EFB1F00B
:10630C00000E1200BCECB1F001012995020E286FB1
:10631C000F0E1200BCECB1F001012995000E286F94
:10632C000F0E1200DBECB1F0D8ECB1F0A6ECB1F032
:10633C00120001012551B7ECB1F01FECB0F01200C6
:10634C0001012995000E286F0F0E12003D01739F5D
:10635C00000E796F78851200016E600007F06BFDFE
:10636C001200016E600007F06CFD12003D01739F7E
:10637C007885738F1200000E71ECACF01200DBEC20
:10638C00B1F0090E1200DEECB1F0040E1200DEECDE
:10639C00B1F0030E1200000E3D01796F12003D01A9
:1063AC006C5112003D01739B12003D01748D120063
:1063BC003D01749D12003D016A5112003D01738D27
:1063CC0012003D01739D12003D01799512003D01B3
:1063DC00769912003D01799F1200010E1200020EF7
:0E63EC001200050E1200010E12001000120029
:020000040020DA
:10000000FF0FFF0FFF0FFF0FFF0FFF0FFF0FFF0F80
:020000040030CA
:0A0000008CD5FFF78DCFFFDFFFFF67
:00000001FF
